:100000000C94390A0C94610A0C94610A0C94610AEC
:100010000C94610A0C94610A0C94610A0C94610AB4
:100020000C94610A0C94610A0C9491250C9400269E
:100030000C94610A0C94610A0C94610A0C94610A94
:100040000C94610A0C94610A0C94610A0C94610A84
:100050000C94610A0C94610A0C94610A0C94322885
:100060000C94610A0C94610A0C94610A0C94610A64
:100070000C94610A0C94610A0C94610A0C94610A54
:100080000C94610A0C94610A0C94610A0C94610A44
:100090000C94610A0C94610A0C94610A0C94610A34
:1000A0000C94610A0C94610A0C94610A383838F88F
:1000B000F8F8C0C0C0C0000000F8F8F8FFFFFFFF6C
:1000C000FFFFFFFFFFFFFFFFFFFFFFFFF8F8F80054
:1000D0000000C0C0C0C0F8F8F83838380000000090
:1000E00000000F0F3F3F3F3F3FFFFFFFF0F0F0FFEB
:1000F000FF3F3F3F3F3F3FFFFFF0F0F0FFFFFF3F7D
:100100003F3F3F3F0F0F00000000000000000000D5
:100110000000000000008080808F8F8F7F7F7F7FB6
:100120007FFEFEFEFEFEFE7F7F7F7F7F8F8F8F80B4
:1001300080800000000000000000000000000000BF
:1001400000000000FEFEFFFFFF1F1F1FFEFEFEFE61
:10015000FEFFFFFFFFFFFFFEFEFEFEFE1F1F1FFF55
:10016000FFFFFEFE00000000000000000000000095
:10017000000000001F1F1F1F1F000000E3E3E3E358
:10018000E3E3E3E3E3E3E3E3E3E3E3E30000001FAC
:100190001F1F1F1F000000000000000000000000E3
:1001A000000000000000000000E0E0E0FFFFFF03AF
:1001B000030000000000000303FFFFFFE0E0E00099
:1001C000000000000000000000000000000000002F
:1001D0000000000000000000FCFCFCFFFFFFFFFF30
:1001E000FFFFFFFFFFFFFFFFFFFFFFFFFFFFFCFC25
:1001F000FC00000000000000000000000000000003
:1002000000000000000000007F7F7FFFFFE0E0E0D3
:10021000E0E0FF9F9FFFFFE0E0E0E0FFFFFF7F7F68
:100220007F0000000000000000000000000000004F
:10023000000000000080808080808083837F7F7F3B
:100240007F7F73737373737F7F7F7F8383838080EC
:10025000808080000000000000000000000000001E
:10026000000000C0C0FFFFFF0101010101CECECEA2
:10027000CECEFEFEFEFEFECECECECE0101010101AF
:1002800001FFFFC0C00000000000000000000000EF
:100290000000000F0F0F0F0F0000F0F0F0F1F1F170
:1002A00031313F3F3F3F3F3131F1F1F0F0F000009D
:1002B000000F0F0F0F000000000000000000000002
:1002C0000000000000000000E0E0FFFFFFFFFFFF74
:1002D000000000000000000000FFFFFFFFFFE0E063
:1002E000E00000000000000000000000FCFCF3F350
:1002F000FFFF0F0F0F0FCFCFFCFC0000000000002E
:10030000F0F0FCFCCFCFC3C3C0C03030000080C0D1
:10031000E0E0E0E0E0E0E0E0C0800000003F7FFFE0
:10032000FFF8FFFFFFFFF8FFFF7F3F000000000026
:100330000000000000FFFFFF0000000000000000C0
:1003400000000000000000000000000000000000AD
:10035000FFFFFF000000000000000000F0F0F000D0
:100360000000000000FFFFFF000000000000F0F0B0
:10037000F0FEFEFEFEFEFEF0F0F0000000000000C9
:10038000FFFFFF000000000000F0F0F01F1F1FE063
:10039000E0E00000000303031C1C1CE0E0E01F1F62
:1003A0001FFFFFFFFFFFFF1F1F1FE0E0E01C1C1CE3
:1003B000030303000000E0E0E01F1F1F0000000037
:1003C0000000070707C7C7C7C7C7C73F3F3FFFFFB3
:1003D000FFFFFFFFFFFFFFFFFFFF3F3F3FC7C7C715
:1003E000C7C7C7070707000000000000000000F0B3
:1003F000F0F00E0E0E010101818181FEFEFEFFFF75
:10040000FFFFFFFFFFFFFFFFFFFFFEFEFE81818179
:100410000101010E0E0EF0F0F0000000000000FFE0
:10042000FFFF000000FCFCFC0303030303031F1F8A
:100430001FFFFFFFFFFFFF1F1F1F03030303030334
:10044000FCFCFC000000FFFFFF00000080C0E0E0BB
:10045000C0C0F0E0E0F0C0C0E0E0C08003010001F7
:100460000301000303000103010001030000000079
:100470000000000000000000C0C0C0F8F8F8F8F864
:10048000F8C0C0C0C0C0C0000000000000000000F4
:10049000000000000000000000000000000000005C
:1004A0000000000000808080FFFFFFFFFFFF8181D0
:1004B00081818181FFFFFF8080808080800000003B
:1004C000000000000000F0F0F0000000000000E07C
:1004D000E0E0FCFCFCFFFFFFE3E3E3FFFFFFFFFFC7
:1004E000FFFFFFFFFFFFFFFFFFFFFFFFFFFCFCFC25
:1004F000000000000000030303FCFCFC0707073FAB
:100500003F3F3F3F3F3F3F3FFFFFFFFFFFFFFFFFFB
:10051000FFFFFFFFFFFFFFFFFFFFFFFFFFFFFFFFEB
:10052000C0C0C0000000C0C0C03F3F3F000000008E
:1005300000000000000000007171717171717F7F17
:100540007F0F0F0F8181818F8F8FFFFFFF0F0F0FA5
:100550000101010E0E0E0F0F0F0000000000000041
:10056000000000000000000000000000000000008B
:100570000000000003030303030303030300000060
:10058000000000000000000000000000183C7EE3B6
:10059000C193817FFFFFFF66FCFCFFFFFFFF0F0F92
:1005A000FFFFFFFF0F0FFFFF3F3FFFFFFFFF3F3F3B
:1005B0003F3FFFFFFFFF3F3F819DFFFF7FFFEDEDCF
:1005C000FFFFFF66387CBE7FFFFFEDEDFFFFFF669C
:1005D0004EF1CEC4CBCDE25C0484651F0701000060
:1005E00043F5CAC2C5CAF54A0484651F0701000065
:1005F00000000010303034FCFC34303010000000BB
:10060000182442819985818F8FA199818142241874
:1006100000000010303034FCFC343030100000009A
:10062000182442998581818F8F8185998142241870
:10063000000000E215151D11111D1515E200000046
:100640000000007F78787878787878787F000000EC
:10065000000000E295959D91919D9595E200000026
:100660000000007F7F7F7F7F7F7F7F7F7F00000094
:100670000000C003E007300C9819D81BCC33CC33F2
:10068000CC33CC33D81B9819300CE007C0030000E2
:1006900000008007C00C60186018C00CF807180034
:1006A00030006000C0008001000300060000000070
:1006B00053433A00580045004C5620002F00485044
:1006C0002000444546200041544B20005700530071
:1006D00045004E002D2D2D004B45590024004600AD
:1006E0004850003E0000000000003E5B4F5B3E3E75
:1006F0006B4F6B3E1C3E7C3E1C183C7E3C181C57CE
:100700007D571C1C5E7F5E1C00183C1800FFE7C371
:10071000E7FF0018241800FFE7DBE7FF30483A0640
:100720000E2629792926407F050507407F05253FAC
:100730005A3CE73C5A7F3E1C1C08081C1C3E7F1498
:10074000227F22145F5F005F5F06097F017F0066E2
:1007500089956A606060606094A2FFA29408047E3C
:10076000040810207E201008082A1C08081C2A08EB
:10077000081E101010100C1E0C1E0C30383E3830A5
:10078000060E3E0E06000000000000005F000000A4
:1007900007000700147F147F14242A7F2A122313D2
:1007A00008646236495620500008070300001C22E6
:1007B00041000041221C002A1C7F1C2A08083E0818
:1007C0000800807030000808080808000060600019
:1007D00020100804023E5149453E00427F4000720D
:1007E000494949462141494D331814127F10274584
:1007F0004545393C4A4949314121110907364949A2
:100800004936464949291E000014000000403400C2
:100810000000081422411414141414004122140876
:1008200002015909063E415D594E7C1211127C7F2E
:10083000494949363E414141227F4141413E7F493C
:100840004949417F090909013E414151737F080827
:10085000087F00417F41002040413F017F08142272
:10086000417F404040407F021C027F7F0408107F90
:100870003E4141413E7F090909063E4151215E7FCB
:1008800009192946264949493203017F01033F409E
:1008900040403F1F2040201F3F4038403F63140826
:1008A000146303047804036159494D43007F4141B7
:1008B000410204081020004141417F04020102046A
:1008C0004040404040000307080020545478407FD7
:1008D000284444383844444428384444287F385411
:1008E00054541800087E090218A4A49C787F0804B8
:1008F000047800447D40002040403D007F102844A3
:100900000000417F40007C047804787C080404786F
:100910003844444438FC1824241818242418FC7C37
:1009200008040408485454542404043F44243C401C
:1009300040207C1C2040201C3C4030403C4428107F
:1009400028444C9090907C4464544C4400083641B8
:100950000000007700000041360800020102040296
:100960003C2623263C1EA1A161123A4040207A3841
:1009700054545559215555794121545478412155A4
:1009800054784020545579400C1E527212395555F6
:100990005559395454545939555454580000457CCC
:1009A000410002457D420001457C40F0292429F0A8
:1009B000F0282528F07C545545002054547C547C64
:1009C0000A097F4932494949323248484832324A55
:1009D0004848303A4141217A3A42402078009DA06F
:1009E000A07D39444444393D4040403D3C24FF24EF
:1009F00024487E4943662B2FFC2F2BFF0929F62024
:100A0000C0887E090320545479410000447D413060
:100A100048484A32384040227A007A0A0A727D0DEC
:100A200019317D2629292F28262929292630484DA4
:100A30004020380808080808080808382F10C8ACF3
:100A4000BA2F102834FA00007B000008142A142260
:100A500022142A14089500220095AA005500AAAA7B
:100A600055AA55AA000000FF00101010FF00141432
:100A700014FF001010FF00FF1010F010F0141414F9
:100A8000FC001414F700FF0000FF00FF1414F4042E
:100A9000FC141417101F10101F101F1414141F0023
:100AA000101010F0000000001F101010101F101088
:100AB0001010F010000000FF101010101010101097
:100AC00010FF10000000FF140000FF00FF00001FD7
:100AD00010170000FC04F414141710171414F40475
:100AE000F40000FF00F714141414141414F700F7A2
:100AF000141414171410101F101F141414F41410CD
:100B000010F010F000001F101F0000001F14000064
:100B100000FC140000F010F01010FF10FF1414146B
:100B2000FF141010101F00000000F010FFFFFFFF67
:100B3000FFF0F0F0F0F0FFFFFF0000000000FFFF0B
:100B40000F0F0F0F0F38444438447C2A2A3E147E7E
:100B500002020606027E027E026355494163384462
:100B6000443C04407E201E2006027E020299A5E736
:100B7000A5991C2A492A1C4C7201724C304A4D4DD1
:100B8000303048784830BC625A463D3E49494900B9
:100B90007E0101017E2A2A2A2A2A44445F444440D5
:100BA000514A444040444A51400000FF0103E08064
:100BB000FF000008086B6B083612362436060F0952
:100BC0000F06000018180000001010003040FF0150
:100BD00001001F01011E00191D1712003C3C3C3C86
:100BE0000000000000F0F89C8E8783878E9CF8F050
:100BF0000000FEFF0303030303070EFCF80000FEE2
:100C0000FF0303030303070EFCF80000FFFF0000CF
:100C10000000000000FFFF0000FEFF83838383834A
:100C2000C7EE7C380000F8FC0E07030303070EFC38
:100C3000F800003F7FE0C08080C0E07F3FFFFF0101
:100C4000010101010101FFFF0000FFFF0C0C0C0C72
:100C50001C3E77E3C100007FFFC0C0C0C0C0E07091
:100C60003F1F00001F3F70E0C0C0C0E0703F1F008A
:100C7000007FFFC1C1C1C1C1E3773E1C00001F3F1F
:100C800070E0C0C0C0E0703F1F000000000001FF26
:100C9000FF01000000D5F08D14A1C881CFD9F1AFBC
:100CA0002000000000000000000000000000000024
:100CB0000000000000000000000000000000000034
:100CC0000000000000000000000000000000000024
:100CD0000000000000000000000000000000000014
:100CE0000000000000000000000000000000000004
:100CF00000000000000000000000000000000000F4
:100D000000000000000000000000000000000000E3
:100D100000000000000000000000000000000000D3
:100D200000000000000000000000000000000000C3
:100D300000000000000000000000000000000000B3
:100D40000000000000000000000000000000E03093
:100D50001010101010101010101010101010101093
:100D60001010101010101010101010101010101083
:100D70001010101030E00000000000000000000023
:100D80000000000000000000000000000000000063
:100D90000000000000000000000000000000000053
:100DA0000000000000000000000000000000000043
:100DB0000000000000000000000000000000000033
:100DC0000000000000000000000000000000FF0024
:100DD000000000000000000003FFFFFFFF0300030E
:100DE00003FFFF7FFEF8F8C0C0F87E7EFFFFFF0321
:100DF0000300000000FF00000000000000000000F1
:100E000000000000000000000000000000000000E2
:100E100000000000000000000000000000000000D2
:100E200000000000000000000000000000000000C2
:100E300000000000000000000000000000000000B2
:100E40000000000000000000000000000000FF00A3
:100E50000000001C7C7CFCE0E0FF7F7F1F0000E0C6
:100E6000E0FFFFE00007070F0703E0E0FFFFFFE000
:100E7000E000000000FF0000000000000000000093
:100E80000000000000000000000000000000000062
:100E90000000000000000000000000000000000052
:100EA0000000000000000000000000000000000042
:100EB0000000000000000000000000000000000032
:100EC0000000000000000000000000000000FF0023
:100ED0000000C4E464646404C4E46464E4C404E43A
:100EE000E4C404C4E4E404E46464646404C4E46442
:100EF0006464000000FF000000000000000000002B
:100F000000000000000000000000000000000000E1
:100F100000000000000000000000000000000000D1
:100F200000000000000000000000000000000000C1
:100F300000000000000000000000000000000000B1
:100F400000000000E0F0F030F0F030F00000FF00B2
:100F50000000070F08090F000F0F0202020F000F19
:100F60000F0103010F0F000F0909090800090B0BFE
:100F70000B07000000FF0000F030F0F030F0F0E070
:100F80000000000000000000000000000000000061
:100F90000000000000000000000000000000000051
:100FA0000000000000000000000000000000000041
:100FB0000000000000000000000000000000000031
:100FC00000000000070F0F07070F0F070000070CB6
:100FD0000808080808080808080808080808080891
:100FE0000808080808080808080808080808080881
:100FF000080808080C070000070F0F07070F0F0766
:1010000000000000000000000000000000000000E0
:1010100000000000000000000000000000000000D0
:1010200000000000000000000000000000000000C0
:1010300000000000000000000000000000000000B0
:1010400000000000000000000000000000000000A0
:101050000000000000000000000000000000000090
:101060000000000000000000000000000000000080
:101070000000000000000000000000000000000070
:101080000000000000000000000000000000000060
:101090000000000000000000000000000000000050
:1010A0000000000000000000000000000000001828
:1010B000F8F8F8F818181878F0F0E018F8F8F8F8D8
:1010C000180018F8F8180818F8F878F8F8E098F800
:1010D000F8180880E0F0F838181818387870000010
:1010E00018F8F8F8F898D8F838786000E0F0F03898
:1010F00018181838F0F0E00018F8F878F8F8E098C8
:10110000F8F81808000000000000000000000000CF
:10111000000000000000000000000000000000309F
:101120003F3F3F3F3030303E1F1F0700071F3F3F0C
:101130003030303F1F0000303F3F3020030F1F3F53
:101140003F0000010F1F3F383030333F3F3F030166
:10115000303F3F3F3F31373738381C070F1F3F388C
:10116000303030381F1F0700303F3F3020030F1F43
:101170003F3F0000000000000000000000000000F1
:10118000000000000000000000000000000000005F
:1011900000000000001C7E6341637F3E417F7F5D55
:1011A0001F03000000366F4D5D7F38417F7F094986
:1011B0007F7F4060785F5F7E70417F7F41637F1EED
:1011C0001C7E6341637F3E033F7D7F3F7D3F070180
:1011D000366F4D5D7F380000004667717F6F2000DD
:1011E00000000000000000000000000000000000FF
:1011F00000000000000000000000000000000000EF
:1012000000000000000000000000000000000000DE
:1012100000000000000000000000000000000000CE
:1012200000000000000000000000000000000000BE
:1012300000000000000000000000000000000000AE
:10124000000000000000000000000000000000009E
:10125000000000000000000000000000000000008E
:1012600000003E004245535420003E004F464600D9
:101270004F4E004D555349432000535441525400A2
:10128000C4000000DC000000F70006011501260183
:1012900000004A015D01000088010000B801D20190
:1012A000EE0100002A024B026E029302BA02000015
:1012B000100300007003904000FA8000FA903D0097
:1012C000FA8000FA903E00FA8000FA903900FA8025
:1012D00000FA9040914300FA808100FA903D9140DD
:1012E00000FA808100FA903E914100FA808100FA74
:1012F0009039913700FA808100FA903C01F4809097
:101300003E00FA80904000FA80904500FA8000FA92
:10131000904500FA8000FA9045913C00FA80819156
:101320003E00FA819043914000FA8081914300FA97
:1013300081904100FA80904000FA80903B00FA8052
:10134000903E00FA80F056494C4C005741520054F0
:101350004846004D4147450041204F4B2042004246
:1013600041534500444546205357440041544B20C7
:1013700053544C004850204D414700434C41535377
:1013800000301030101030306C044C042C030C036F
:10139000EC02CC01AC005350430041544B00454893
:1013A00020002F004850200032352048502B0032BA
:1013B00030204445460032302041544B003520480F
:1013C00045414C00464F554E54004850202B3200AA
:1013D000444546202B310041544B202B31004C56C4
:1013E000205550004120525354204220484F4D4533
:1013F0000047414D45204F56455200080B00020260
:10140000020000090400000102020000052400108F
:101410000105240101010424020605240600010738
:1014200005810310004009040100020A00000007C2
:101430000502024000000705830240000004030982
:101440000412010002EF0201404123368000010135
:1014500002030141726475696E6F204C4C43004178
:10146000726475696E6F204C656F6E6172646F0097
:10147000AF2811241FBECFEFDAE0DEBFCDBF12E0F0
:10148000A0E0B1E0E8ECFEE602C005900D92AE31BE
:10149000B107D9F727E0AEE1B2E001C01D92A03E4E
:1014A000B207E1F71AE0C9E3DAE004C02197FE01D0
:1014B0000E945C37C833D107C9F70E94CC280C942E
:1014C00062370C940000809136018E5F8093360164
:1014D00090913501981710F49093360108954F922A
:1014E0005F926F927F928F929F92AF92BF92CF92B4
:1014F000DF92EF92FF920F931F93CF93DF93FB0145
:10150000E00FF11D1E161F060CF08FC06034710530
:101510000CF08BC0DB0177FF04C0AA27BB27A61BFA
:10152000B70BA770BB27EB0177FD2796E3E0D595B6
:10153000C795EA95E1F777FF07C0219768E070E06B
:10154000FB01EA1BFB0BDF01E02EE694E694E69438
:10155000F12C077019F0FFEFEF1AFF0A30E08A0153
:10156000AE015695542F442757954795480F591F5C
:1015700044575C4FBE01E0E8F0E05F01A81AB90AE9
:1015800088E090E03C016A1A7B0A6F3F8FEF780792
:101590000CF43BC090E080E04A01E0E88E0E911C24
:1015A0006F3F760709F452C0FC01E00FF11FE49190
:1015B0006A01C80ED91EF0E02F010A2E01C0440CAA
:1015C0000A94EAF7F6015080452840821097B1F05E
:1015D0006730710599F0F801E80FF91FE491640193
:1015E000C80ED91EF0E02F01062C02C05594479476
:1015F0000A94E2F7F601508045284082019682174E
:1016000093071CF4A816B90659F66F5F7F4F020FB7
:10161000131F40585F4FCB018C1B9D0B8E159F05F0
:1016200024F46830710509F0B0CFDF91CF911F919C
:101630000F91FF90EF90DF90CF90BF90AF909F9071
:101640008F907F906F905F904F900895109709F062
:10165000C2CFD4CFECE8F3E0A0E0B8E000800EBC4D
:101660008111012C1197A0FDFDCF0192B9F70DB4A6
:101670000895FC0180918B03882311F13FB7F89402
:1016800082E08093E9002091F200822F90E018160A
:10169000190614F481E090E0882339F0289844E694
:1016A00040938A034091F1004083222339F0209136
:1016B000F200211103C02BE62093E8003FBF0895FC
:1016C0008FEF9FEF08952FB7F89483E08093E900A0
:1016D0009091E800892F807295FF04C09091F200EC
:1016E00080E4891B2FBF08958091820381110DC072
:1016F00082E080937E0384E080937F0310928103D5
:101700001092800381E0809382038EE793E0089536
:10171000CF93DF931F92CDB7DEB76983DC01ED91E4
:10172000FC910280F381E02D41E050E0BE016F5F4B
:101730007F4F09950F90DF91CF91089583E08093BB
:10174000E9008091F200882319F08AE38093E80091
:1017500008950E94630B90E00895CF93DF931F924A
:10176000CDB7DEB7FC018485958597FD08C02FEFC6
:101770003FEF358724870F90DF91CF910895CE01F9
:1017800001960E94390B019719F4898190E0F3CFFB
:101790008FEF9FEFF0CF0F931F93CF93DF931F92A5
:1017A000CDB7DEB78C01FC018485958597FF0BC012
:1017B000CE0101960E94390B019771F4898190E066
:1017C000F80195878487F801848595850F90DF91CE
:1017D000CF911F910F9108958FEF9FEFF1CFFC01F3
:1017E0008485958597FD0BC09FB7F89482E0809320
:1017F000E9008091F2009FBF90E0019608959FB7A5
:10180000F89482E08093E9008091F2009FBF90E01D
:101810000895409178035091790320917603309197
:10182000770342175307B4F49091E8009570E1F301
:101830009091E80092FD19C08093F10080917803A7
:101840009091790301968F739927892B19F48EEF64
:101850008093E800809178039091790301969093AA
:1018600079038093780381E0089580E00895DF9202
:10187000EF92FF920F931F93CF93DF93D82E8A019D
:10188000EB017B01E40EF51ECE15DF0559F0D7FE06
:1018900012C0FE0184910E94090C21968111F4CF9F
:1018A0000FEF1FEFC801DF91CF911F910F91FF90B4
:1018B000EF90DF9008958881EECF0F931F93CF9321
:1018C000DF931F92CDB7DEB782E0898342E450E018
:1018D0006BEF73E180E80E94370C0E94740BDC010F
:1018E00012960D911C910115110589F0D801ED9109
:1018F000FC910280F381E02DBE016F5F7F4FC80134
:10190000099597FD04C0F80100851185ECCF898108
:101910000F90DF91CF911F910F910895615030F09A
:101920002091F100FC0120830196F8CF289884E6ED
:1019300080938A0308953FB7F89480917203909141
:101940007303A0917403B091750326B5A89B05C0DD
:101950002F3F19F00196A11DB11D3FBFBA2FA92F2E
:10196000982F8827BC01CD01620F711D811D911D2B
:1019700042E0660F771F881F991F4A95D1F7089597
:101980008F929F92AF92BF92CF92DF92EF92FF928F
:101990006B017C010E949B0C4B015C01C114D104C2
:1019A000E104F104B9F00E949B0C681979098A09D5
:1019B0009B09683E73408105910580F321E0C21ABE
:1019C000D108E108F10888EE880E83E0981EA11C7A
:1019D000B11CE4CFFF90EF90DF90CF90BF90AF901D
:1019E0009F908F9008958F929F92AF92BF92CF92C7
:1019F000DF92EF92FF920F931F93CF93DF936C01CF
:101A00007B018A0180913401882309F45CC08091B4
:101A10008B03882309F457C080917D0380FF05C0A4
:101A20008091E00082608093E000E801B12C8AEFB1
:101A3000A82E93E0892E2AE3922E209711F4BB2042
:101A4000D9F10E94630B81110AC0AA94AA20D9F18E
:101A500061E070E080E090E00E94C00CEECF8C1757
:101A60001D0611F00CF08C2F9FB7F8948092E900BE
:101A70002091E80025FD02C09FBFDFCF282F30E076
:101A8000C21BD30BF701815020F041914093F1002C
:101A9000FACFE20EF31EBB2021F09092E800B12CA9
:101AA000EBCF8091E80085FDE7CF9092E800BB2462
:101AB000B394209709F3F3CF5D9884E680937C0379
:101AC000101611063CF081E090E0F60193838283CA
:101AD00010E000E0C801DF91CF911F910F91FF90BE
:101AE000EF90DF90CF90BF90AF909F908F90089530
:101AF000AF92BF92CF92DF92EF92FF920F931F931C
:101B0000CF93DF936C017B018B01040F151FEB0159
:101B10005E01AE18BF08C017D10759F06991D60110
:101B2000ED91FC910190F081E02DC6010995892B82
:101B300079F7C501DF91CF911F910F91FF90EF9041
:101B4000DF90CF90BF90AF9008952D9A0895BC017B
:101B500090E080E00C94C00C8FB18095807F669BF4
:101B600088601C9B846008953E983F9808953E9A33
:101B70003F9A089580E0ECE8F3E081118FEF0024B4
:101B800081938193819381930394D1F710926103A0
:101B90001092600310926303109262030895909173
:101BA0002703982329F490912803982381E009F4CE
:101BB00080E0089580E00C942A0B6034710508F0F1
:101BC0003EC0480F592F511D14161506C4F5803814
:101BD0009105ACF597FF02C090E080E041385105D7
:101BE00014F040E850E0481BFB0133E0F595E79521
:101BF0003A95E1F7F695FE2FEE27F795E795E80F72
:101C0000F91FE457FC4F6770772781E090E001C02F
:101C1000880F6A95EAF7382F213041F4415078F067
:101C20008191DF011197832B8C93F8CF80954150E0
:101C300030F09191DF01119798239C93F8CF08958C
:101C40002F923F924F925F926F927F928F929F92CC
:101C5000AF92BF92CF92DF92EF92FF920F931F93BA
:101C6000CF93DF93CDB7DEB72E970FB6F894DEBFD4
:101C70000FBECDBF5B015E874D8769012617370711
:101C80000CF0F9C0E616F7060CF40CC13A2D2B2D1A
:101C90005601C32ED22E382F292F8D859E853D8744
:101CA0002E87AE14BF04B1F52D853E852817390760
:101CB00034F4382F292F8D859E853D872E87081770
:101CC000190744F04D855E854017510714F41E87AF
:101CD0000D878C014D854F5F401B21E0B501C80188
:101CE0002E960FB6F894DEBF0FBECDBFDF91CF9119
:101CF0001F910F91FF90EF90DF90CF90BF90AF902A
:101D00009F908F907F906F905F904F903F902F901B
:101D10000C94DD0D302F212F8C01832F922F3E2D1F
:101D20002F2D7501A32EB22E2D853E85201B310B44
:101D300038872F83A6014E195F095A8749873C01CE
:101D4000601A710A95012E193F093A832983AC0163
:101D50002D853E85421B530B5C834B83A5014C199B
:101D60005D095C874B87CA14DB0409F43FC0C601D8
:101D700001979E838D834701512C412C312C212CBE
:101D80002D813E8128153905A4F1C10169857A8527
:101D90000E944137FB01E00FF11FC20169817A8186
:101DA0000E944137600F711F4F815885240E351EE8
:101DB000460C571C6E177F071CF49E2FFB01692FE2
:101DC0006F5F462F4E1B21E0B401CF010E94DD0D55
:101DD0005FEF851A950AD4CF3D852E859E878D8726
:101DE000832F922F3A2D2B2D560169C0DE82CD8292
:101DF000C2CFC4018C199D092B813C81829F600157
:101E0000839FD00C929FD00C1124C4018E199F097E
:101E1000869D7001879DF00C969DF00C1124A814EE
:101E2000B9040CF44FC0C6016B857C850E94413714
:101E3000ED85FE85E60FF71FC70169817A810E9453
:101E40004137600F711F4B815C81C40ED51EE60CBB
:101E5000F71C6E177F071CF49E2FFB01692F6F5F25
:101E6000462F4E1B21E0B401CF010E94DD0D5FEF34
:101E7000851A950AD4CFE216F3060CF012CFE616B7
:101E8000F7060CF4A9CF302F212F0D851E859E87D4
:101E90008D87832F922F3C2D2D2D6B015701E32E23
:101EA000F22EF4CEE216F3060CF43ECF302F212FA3
:101EB0000D851E853D872E873E2D2F2D7601C32E45
:101EC000D22E32CF2E960FB6F894DEBF0FBECDBF06
:101ED000DF91CF911F910F91FF90EF90DF90CF9006
:101EE000BF90AF909F908F907F906F905F904F903A
:101EF0003F902F90089580389105B8F460347105B3
:101F0000A0F420E191E061FD94E060FD990F62FD95
:101F10009295687F269FD0011124A80FA457BC4F2B
:101F20008C9140FF03C0892B8C9308959095892351
:101F3000FBCF2F923F924F925F926F927F928F9240
:101F40009F92AF92BF92CF92DF92EF92FF920F9348
:101F50001F93CF93DF9300D000D000D0CDB7DEB772
:101F6000342F36951C01231A3108A22EB12CCB0137
:101F70008A199B099E838D83712C612C4424439480
:101F8000512C842E912C6A147B0409F483C08D811A
:101F90009E810897C89708F06DC0C30154E0880F70
:101FA000991F5A95E1F7B5010E942D37F62ECB0106
:101FB000887F99279A8389836770C20102C0880F3E
:101FC000991F6A95E2F79C838B83D12CC12CC8148E
:101FD000D90409F44FC091012C0D3D1D2038310565
:101FE00008F044C0C60143E0880F991F4A95E1F705
:101FF000B4010E942D37A62FEE2011F0A7E0A61BFA
:10200000E981FA81EA0FF11DE00FF11FE491F0E0A0
:102010008B819C81E823F92341E0EF2BA9F59FEF09
:10202000B2E0BA0F8F2D890F8031E8F4482F50E0CD
:10203000487F55278770B20102C0660F771F8A95C7
:10204000E2F78FEF8A0F883058F4FA01E80FF11D9C
:10205000E00FF11FE491F0E0E623F723EF2B99F472
:102060008F5FB813F0CF9F5F9230E1F69FEFC91AF0
:10207000D90AADCF8FEF681A780A8D819E810196BB
:102080009E838D8380CF40E06D817E81C9010E9457
:102090007B0FECCF26960FB6F894DEBF0FBECDBFF8
:1020A000DF91CF911F910F91FF90EF90DF90CF9034
:1020B000BF90AF909F908F907F906F905F904F9068
:1020C0003F902F9008952F923F924F925F926F9280
:1020D0007F928F929F92AF92BF92CF92DF92EF92B8
:1020E000FF920F931F93CF93DF9300D000D000D0C7
:1020F000CDB7DEB7522E242F2695821B91099A83E5
:102100008983A52CB12C1B012A183B083E822D8205
:10211000D12CC12C642E712C50E8852E912CC60137
:10212000B5010E942D37462EF12CE12CC801860FF7
:10213000971F9C838B836E147F0409F449C0298107
:102140003A812E0D3F1D2038310508F03DC0C701F2
:1021500043E0880F991F4A95E1F7B3010E942D379C
:10216000EB81FC814491C401062E02C095958795B0
:102170000A94E2F750E08423952341E0892B09F08B
:102180004EC08FEFA42DA80FAF3FD9F0AC30CCF4E8
:102190009FEFA00FB12FB11D592F560F583070F47B
:1021A000FD017491F40102C0F595E7955A95E2F7A7
:1021B000AF01F0E047235F23452B81F59F5F92300D
:1021C00059F78F5F8230F1F6FFEFEF1AFF0AB3CFB6
:1021D0008CE0C80ED11CED81FE813196FE83ED832B
:1021E0008E2F8219851508F49ACF26960FB6F8948B
:1021F000DEBF0FBECDBFDF91CF911F910F91FF903A
:10220000EF90DF90CF90BF90AF909F908F907F9096
:102210006F905F904F903F902F90089540E06D81B8
:102220007E81C9010E947B0FCFCF2F923F924F92A8
:102230005F926F927F928F929F92AF92BF92CF9256
:10224000DF92EF92FF920F931F93CF93DF93CDB75F
:10225000DEB728970FB6F894DEBF0FBECDBF6D3046
:10226000D9F0309028014090600350906103832D95
:1022700090E098878F836A3051F510926303109233
:10228000620323E0880F991F2A95E1F7480E591E33
:10229000509261034092600381E090E028960FB66F
:1022A000F894DEBF0FBECDBFDF91CF911F910F918C
:1022B000FF90EF90DF90CF90BF90AF909F908F9066
:1022C0007F906F905F904F903F902F9008959091E6
:1022D00027019B83A0906203B0906303E5E06E9FAB
:1022E000B0011124CB018B51994F3C01650119823A
:1022F0009981212C953029F0C3010196F301249096
:102300003C014201F8E0FA8320FE1DC02B812C83A2
:1023100010E000E00315D0F4F601E00FF11FFE839A
:10232000ED83F12CE12CE31480F5B4016E0D7F1DDB
:102330004C818D819E810E947B0FFFEFEF1AFF0A77
:10234000F2CF1C82E5CF8B818111FBCF26942A81AD
:1023500021502A838F819885880E991E2111D4CF10
:1023600099819F5F9983EF81F885CE0EDF1E9630AD
:1023700009F0BECFC501F9813F9E800D911D11244A
:10238000909363038093620387CF0F5F1F4FC2CF89
:102390000F931F93CF93DF938C01D0E0C0E0F8013F
:1023A000EC0FFD1F6491662341F08CED97E00E94D5
:1023B0001511892B11F02196F2CFCE01DF91CF912B
:1023C0001F910F910895DF92EF92FF920F931F9349
:1023D000CF93DF937C01D22E8B01040F111DEB01F3
:1023E00077FF02C0D0E0C0E0C8010134110514F04D
:1023F00080E490E0C817D9073CF44D2DBE01C70119
:102400000E947B0F2196F0CFDF91CF911F910F910A
:10241000FF90EF90DF900895CF92DF92EF92FF92BE
:102420000F931F93CF93DF936B01122FEC017C016D
:10243000E40EF11CCE15DF0544F4202F412FB60128
:10244000CE010E94E3112196F5CFDF91CF911F912C
:102450000F91FF90EF90DF90CF900895CF92DF9291
:10246000EF92FF920F93CF93DF936C017B01C42F08
:10247000D22F202F0E94DD0DB7016D0F711D61500D
:102480007109202F4C2FC6010E94DD0D202F4D2FEA
:10249000B701C6010E94E311C6018C0F911D202FC8
:1024A0004D2FB7010197DF91CF910F91FF90EF90E2
:1024B000DF90CF900C94E3112F923F924F925F9256
:1024C0006F927F928F929F92AF92BF92CF92DF9244
:1024D000EF92FF920F931F93CF93DF9300D01F9241
:1024E000CDB7DEB79B838A837B016A0109838901AB
:1024F000061B170B17FF03C0119501951109460123
:102500008A819B81881A990A97FE03C091948194CD
:102510009108801691065CF49C2D8D2D6901292F60
:10252000382F9A818B81FB82EA82E92EF82E8A81EC
:102530009B81C816D9065CF49E2D8F2D7901292F19
:10254000382F9A818B81DB82CA82C92ED82E160140
:102550008A819B81281A390A29014E185F0857FE83
:1025600003C0519441945108310137FE03C09FEFDD
:10257000691A790A759467948FEFE216F3060CF4E2
:1025800081E0A82E880FBB088A819B81C816D906D6
:10259000CCF04981BC01C701801691061CF0B7013F
:1025A0008A819B810E947B0F6418750877FE04C0A6
:1025B000EA0CFB1C620C731C8A819B8101969B8335
:1025C0008A83E2CF0F900F900F90DF91CF911F91F0
:1025D0000F91FF90EF90DF90CF90BF90AF909F90C2
:1025E0008F907F906F905F904F903F902F900895C5
:1025F0000F931F93CF93DF93C82FCB01042F122F7C
:10260000D0E022E130E03093630320936203D09363
:102610006103C09360030E94C811011312C088E0D7
:1026200090E09093630380936203D0936103C0931F
:10263000600383EE96E0DF91CF911F910F910C9490
:10264000C811DF91CF911F910F9108956F927F92E2
:102650008F929F92BF92CF92DF92EF92FF920F9351
:102660001F93CF93DF93B42E49013801C62FD0E0DA
:10267000E82EF12C01E025E0BE01C7010E942E12D8
:1026800061147104F1F0CB2CD12CD6011297940176
:102690000E945537930150E040E00E94D734422F0A
:1026A00081E0C81AD1082C151D0414F04EEF4B0D13
:1026B000BE016F5F7F4F01E023E0C70101960E94DA
:1026C0000C12DF91CF911F910F91FF90EF90DF904F
:1026D000CF90BF909F908F907F906F9008952F9292
:1026E0003F924F925F926F927F928F929F92AF92A2
:1026F000BF92CF92DF92EF92FF920F931F93CF93EF
:10270000DF9300D000D000D0CDB7DEB74B0158E04A
:10271000859F90011124F901E95CFE4F46805780A6
:10272000449DC001459D900D112464E670E00E9417
:102730004137362E86E0681710F476E0372EF9011F
:10274000E95CFE4F8481958197FD0196959587956B
:10275000F901E95CFE4F20813181820F931F232D07
:102760002695AC01421B51095A834983828193818A
:10277000480E591E51E0451A5108A32CB12C4A1895
:102780005B088201D12CC12C612C60E8762EC80137
:102790000897C89708F05FC0C601B5010E942D37A1
:1027A000262E7727660F771FC401860F971F9C83FD
:1027B0008B8349815A815E834D83F12CE12C8D817D
:1027C0009E818038910508F037C0C701B5010E948D
:1027D0002D37EB81FC8125913491C301062E02C077
:1027E000969587950A94E2F78223932341E0892BFB
:1027F00009F055C02FEF822D820F8031D0F490E088
:10280000880F991F880D991D3FEF732F760F703138
:1028100068F4FC0145915491F30102C0F695E795E7
:102820007A95E2F74E235F23452BC1F53F5F3230A7
:1028300061F72F5F2230F9F64D815E814F5F5F4F68
:102840005E834D8350E1E50EF11C842F9981891B35
:10285000831508F4B4CF0F5F1F4F40E1C40ED11CA5
:10286000802F8419831508F492CF26960FB6F8941A
:10287000DEBF0FBECDBFDF91CF911F910F91FF90B3
:10288000EF90DF90CF90BF90AF909F908F907F9010
:102890006F905F904F903F902F90089540E0B80167
:1028A0008D819E810E947B0FC7CFBF92CF92DF9216
:1028B000EF92FF920F931F93CF93DF938C019B01B5
:1028C000E42EDC011696BC9016971796FC908B2D83
:1028D0009F2D63E070E00E944137C62F673108F0FA
:1028E000C6E1CA3008F4CAE0DC2FD695F801C080F2
:1028F000D180F901A081B181EE2071F0F8018481CD
:102900009581C80ED91EF1E0CF1AD108F901848152
:102910009581A80FB91F1197AC19BD0923E030E0CC
:102920000E94553728E030E040E050E00E94AD348E
:10293000C601820F931F6B2D7F2D77FF02C06F5F43
:102940007F4F75956795D80112964D915C91640FF4
:10295000751F6D0F711D2091550300EE15E024FDCC
:1029600002C000ED15E02C2F4D2F0E94990FDF9132
:10297000CF911F910F91FF90EF90DF90CF90BF907C
:1029800008952F923F924F925F926F927F928F9213
:102990009F92AF92BF92CF92DF92EF92FF920F93EE
:1029A0001F93CF93DF93CDB7DEB729970FB6F89477
:1029B000DEBF0FBECDBF742E1901242F2695821BBA
:1029C00091099A838983842F90E09B01281B390BFE
:1029D0003987288710E0B12CA12C612C542E492E68
:1029E0004801671409F4A1C0888599850897C8979C
:1029F00008F08AC0C501652D742D0E942D376B83A8
:102A0000CB0153E0959587955A95E1F78F719927FA
:102A1000809F9001819F300D909F300D11243D8348
:102A20002C83677081E090E002C0880F991F6A953F
:102A3000E2F79F838E83E980FA80D12CC12C90E845
:102A4000E916F10408F055C0C601652D742D0E94E9
:102A50002D37EC81FD81E60FF11DE20DF31DE491B0
:102A6000F0E02E813F81E223F32341E0EF2B09F0D8
:102A700056C08FEF9B81980F97FD37C0292F092EE5
:102A8000000C330B2815390584F5292F30E043E07D
:102A9000359527954A95E1F7209FA001219F500D7C
:102AA000309F500D1124977021E030E002C0220FBA
:102AB000331F9A95E2F79FEFE92FE60FE7FD12C06B
:102AC000AE2F0E2E000CBB0BA815B9055CF4E40F5D
:102AD000F52FF11DE20DF31DE491F0E0E223F32365
:102AE000EF2BE1F49F5F923039F78F5F823009F06E
:102AF000C1CF3FEFE31AF30AC00ED11E8E2D99818C
:102B0000891B871508F49BCF6394288539852F5F2F
:102B10003F4F39872887A00EB11E63CF40E06885FC
:102B20007985C7010E947B0FE4CF29960FB6F894F0
:102B3000DEBF0FBECDBFDF91CF911F910F91FF90F0
:102B4000EF90DF90CF90BF90AF909F908F907F904D
:102B50006F905F904F903F902F900895EF92FF926B
:102B60000F931F93CF93DF93EB017A01E22F811133
:102B700017C0822F90E0880F991F63E070E00E94D9
:102B80004137462F04EC15E02E2FB701CE010E94ED
:102B90006310DF91CF911F910F91FF90EF900895F7
:102BA000813061F4822F90E0880F991F63E070E01C
:102BB0000E944137462F0CE815E0E6CF823061F4E1
:102BC000822F90E0880F991F63E070E00E944137E8
:102BD000462F08EB15E0D8CF00E128E935E04E2F6D
:102BE000B701CE010E94C114D4CFEF92FF920F9390
:102BF000CF93DF937B01042F98E0899FF00111248C
:102C0000DF01A95CBE4F1696CD91DC912C9FC001CF
:102C10002D9F900D112464E670E00E944137462FED
:102C2000663008F446E0DF01A95CBE4F12966D9154
:102C30007C9113976C0F7D1F6150710914968D91D3
:102C40009C9197FD019695958795E95CFE4F0190C3
:102C5000F081E02D97018E0F9F1F0E94C114DF911C
:102C6000CF910F91FF90EF9008952F923F924F9246
:102C70005F926F927F928F929F92AF92BF92CF920C
:102C8000DF92EF92FF920F931F93CF93DF93CDB715
:102C9000DEB7AE970FB6F894DEBF0FBECDBFFC0116
:102CA000DB0116960D911C9117971E830D83C6802C
:102CB000D78020803180228133813A8329836D91AE
:102CC0007C91119778876F8312968D919C911397C1
:102CD0009C838B835801A80EB91E49018C0C9D1C46
:102CE000442381F084819581280E391E91E0291AB0
:102CF000310814968D919C91680F791F615071096C
:102D000078876F8375010F8118852B813C81A8011D
:102D100069817A81C1010E94200E740181019501AF
:102D20004F81588569817A81C1010E94200E00E09F
:102D30002B813C814F81588569817A81C1010E9434
:102D40005C1295014F8158856B817C81CA010E947C
:102D50005C129401A101B5018F8198850E945C12DB
:102D600029813A81A101B401C1010E945C1214E0E1
:102D7000BB24B39495E0492E512C612C712C8B2CE3
:102D8000912C9401AD81BE810E945537A30192011F
:102D90000E94AD34EB80FC80E20EF31E9401D6015C
:102DA0000E945537A30192010E94AD3469817A8156
:102DB000620F731F00E097014F815885C1010E9487
:102DC0005C12B3941150D9F60D2C000CEE08FF08DC
:102DD00026013701440C551C661C771C0D811E8191
:102DE000C801110FAA0BBB0B4C015D01880C991C8B
:102DF000AA1CBB1CA701960112E0220F331F441F1F
:102E0000551F1A95D1F72F8B388F498F5A8FAC01E8
:102E1000BD0102E0440F551F661F771F0A95D1F7C9
:102E20004F87588B698B7A8B6F817885CB01770FB1
:102E3000AA0BBB0BA101032C000C660B770B8C01BA
:102E40009D01041B150B260B370B0B8F1C8F2D8F31
:102E50003E8F86E0000F111F221F331F8A95D1F786
:102E60000FA318A729A73AA710E0C301B20128E2CF
:102E700030E040E050E00E94AD3469817A81620F19
:102E8000731F78876F838F89988DA98DBA8D840D74
:102E9000951DA61DB71D8B8B9C8BAD8BBE8BBC016E
:102EA000CD0128E230E040E050E00E94AD34A9813D
:102EB000BA81A20FB31FBE83AD832F85388949899C
:102EC0005A89280D391D4A1D5B1D2B873C874D876C
:102ED0005E87312F3072432F50E0405C5F4F5EA71A
:102EE0004DA76A01550FEE08FF08A70196016B8DEB
:102EF0007C8D8D8D9E8D0E9411372B013C01C5016B
:102F0000B40128E230E040E050E00E94AD346B8133
:102F10007C81260F371F032E000C440B550B6F814D
:102F20007885CB01770FAA0BBB0B281B390B4A0BFB
:102F30005B0BDA01C90166E0880F991FAA1FBB1F4E
:102F40006A95D1F78BA39CA3ADA3BEA3C701B6011D
:102F50000E9411374B015C016B857C858D859E85B8
:102F600028E230E040E050E00E94AD34AB81BC810B
:102F70002A0F3B1F032E000C440B550B6D817E81E5
:102F8000CB01770FAA0BBB0B281B390B4A0B5B0B32
:102F9000DA01C90176E0880F991FAA1FBB1F7A9535
:102FA000D1F78F8F98A3A9A3BAA3C701B6010E9436
:102FB00011376B017C01C301B20120E031E040E038
:102FC00050E00E94AD34D101A20FB31FBA87A98788
:102FD000C701B60120E031E040E050E00E94AD348E
:102FE0006D817E81620F731F7CA76BA7C501B40141
:102FF00020E031E040E050E00E94AD346F81788500
:10300000620F731F00E02BA53CA549855A85CA01B4
:103010000E945C128DA59EA5805C9F4F9EA78DA7E8
:103020002FA138A549A55AA5420E531E641E751E30
:103030004BA15CA16DA17EA1840E951EA61EB71E9C
:103040006F8D78A189A19AA1C60ED71EE81EF91E20
:103050008DA59EA58F3F91050CF4ADCF4B885C8864
:103060006D887E882F89388D498D5A8D420E531E6A
:10307000641E751E8B849C84AD84BE844F855889E4
:1030800069897A89840E951EA61EB71E105E103AB5
:1030900009F0EBCEAE960FB6F894DEBF0FBECDBFF3
:1030A000DF91CF911F910F91FF90EF90DF90CF9024
:1030B000BF90AF909F908F907F906F905F904F9058
:1030C0003F902F90089520911E02EDE3F3E090E0F1
:1030D000291771F03281131644F43081381305C07A
:1030E0003181361302C0892F08959F5F3496F0CF47
:1030F0008FEF0895CF93DF93EC01A8E0B1E0E0E01B
:103100009991992321F09D93EF5FE131C9F7F0E0A8
:10311000E85FFE4F108286E180933B03DF91CF9101
:10312000089580912601889FC00111249C01220FDF
:10313000331F820F931F06960895809133038F5F8C
:10314000843018F4809333030895109233038091F0
:1031500022018F5F8093220190911E01981710F435
:103160009093220108954091680350916903609102
:103170006A0370916B03480F591F611D711D4093C5
:1031800068035093690360936A0370936B03089517
:1031900010922C0310922B0310922D0310922E03E9
:1031A00010922F03109230038FEF80931D018093B4
:1031B0001C0110922A031092900010922903109281
:1031C000C0000895CF92DF92EF92FF920F931F936A
:1031D000CF93DF9330913103332379F1022FEA014A
:1031E000162FBC0190E080E00E9416366B017C0136
:1031F00020E030E040E05FE30E94A43620E034E2CB
:1032000044E759E40E940935A70196010E947535EB
:103210000E94E7356150710910932A0380E480937E
:1032200090007093990060939800D0932503C09309
:1032300024030093230310932603DF91CF911F9162
:103240000F91FF90EF90DF90CF90089581110CC007
:1032500084E891E00E947A1823E040EA50E063E0BD
:1032600088E191E00C94E218909136018917B0F052
:10327000109236018AE891E00E947A1826E041E433
:1032800050E065E08AE590E00E94E2188091360106
:10329000811103C087E080936C030895981B90937D
:1032A0003601E8CFCF93DF93C0915C03D0915D03EB
:1032B000C80FD11DD0935D03C0935C030E94911889
:1032C000C817D90798F080916C03833079F4109275
:1032D0005E0386E080936C0325E048E255E064E0FD
:1032E00080E793E0DF91CF910C94E218DF91CF91CA
:1032F0000895CF92DF92EF92FF92CF932091310306
:10330000222329F1C62FBC0190E080E00E941636EE
:103310006B017C0120E030E040E05FE30E94A436D6
:1033200020E034E244E759E40E940935A701960100
:103330000E9475350E94E73561507109C0932A03D8
:1033400080E4809390007093990060939800CF91EF
:10335000FF90EF90DF90CF9008958091310391E03E
:10336000892780933103882349F00E94B70D0E947A
:10337000C8186DE288EE93E00C9479190E94C81881
:103380000C94B40D0F931F93809100019091010153
:10339000A0910201B09103018C019D014DE0000F4D
:1033A000111F221F331F4A95D1F7082719272A27F3
:1033B0003B27D901C80151E1B695A7959795879507
:1033C0005A95D1F7082719272A273B27C901B801A1
:1033D000E5E0660F771F881F991FEA95D1F76027F0
:1033E00071278227932760930001709301018093D6
:1033F0000201909303011F910F910895809324017E
:1034000010923C03109256031092570310923A0305
:103410001092390384E080936C0323E04CEC51E07C
:1034200063E08EE591E00E94E2180E94C21960FFFD
:103430000DC086E08093560381E0809339038FE0CE
:10344000809357038FE891E00C947A1808950F93B6
:103450001F93CF93DF938C01EB010E94C2199E0151
:10346000201B310B2F5F3F4F032E000C440B550BDD
:103470000E94D734C801860F971FDF91CF911F910B
:103480000F910895803170F4603160F490E1690229
:10349000F0011124E15EFD4FE80FF11D87FDFA9563
:1034A0008081089581E00895CF93DF93C0911F013B
:1034B000D09120016C2F8D2F0E94421A8330D9F4B5
:1034C00020E1C29FC0011124815E9D4F8D0F911D8F
:1034D000FC01108281E08093360388EA91E00E942B
:1034E0007A1824E048E255E063E080E793E0DF915A
:1034F000CF910C94E218843011F5F0E1CF9FC00118
:103500001124815E9D4F8D0F911DFC0110828091D1
:10351000580390915903019690935903809358034F
:103520008AE090E00E94B31887E991E00E947A183F
:1035300023E04CE657E062E08CED95E0D8CF853093
:10354000F1F4F0E1CF9FC0011124815E9D4F8D0FFA
:10355000911DFC0110820E94630A81E00E945219B1
:1035600085E090E00E94B3188FE991E00E947A18FC
:1035700024E042E553E064E086E292E0B8CFDF91D8
:10358000CF9108953F924F925F926F927F928F9268
:103590009F92AF92BF92CF92DF92EF92FF920F93E2
:1035A0001F93CF93DF93CDB7DEB7DA950FB6F894BC
:1035B000DEBF0FBECDBF7C01FC0193952FEF2193A1
:1035C0008E179F07E1F780911F0190E1899F90017D
:1035D000112480912001820F932F911DF701E80F94
:1035E000F91F1082898301E0E0E03BE5A32E31E082
:1035F000B32E662463946E0E81E090E08C0F9D1FC5
:103600008E0F911DFC01E0819E2F9F70592E4E2E32
:1036100042948FE04822EE0DFF2DF11D70807394CF
:1036200097E5892E91E0992E2BE5C22E21E0D22E2E
:10363000F40111914F01150DF60161916F01362EC4
:10364000340C632D812F0E94421A811115C0F0E1C4
:103650003F9EB0011124610F711DF701E60FF11DAE
:1036600080818F3F49F47082E1E0F0E0EC0FFD1FB4
:10367000E00FF11D60830F5FA814B904C9F6E62DB1
:103680000611B7CFD3950FB6F894DEBF0FBECDBFEE
:10369000DF91CF911F910F91FF90EF90DF90CF902E
:1036A000BF90AF909F908F907F906F905F904F9062
:1036B0003F900895DF92EF92FF920F931F93CF9365
:1036C000DF93D82FD62E0BE511E087E5E82E81E0B9
:1036D000F82EC0E0F80161918F01F70181917F011F
:1036E0006D0D8D0F0E94421A811101C0CF5FF1E074
:1036F0000F351F0779F78C2FDF91CF911F910F9115
:10370000FF90EF90DF9008955F926F927F928F927B
:103710009F92AF92BF92CF92DF92EF92FF920F9360
:103720001F93CF93DF93582E5B0130E5632E6EE03D
:1037300070E081E090E00E94271A8C016EE070E05A
:1037400081E090E00E94271A7C01EC01DD276801EE
:10375000DD2443E0682F802F541208C00E945A1BBA
:1037600077247394823040F0712C06C00E945A1B5B
:10377000772473948330C0F7CE0124E0880F991F1B
:103780002A95E1F79C012C0D3D1DA901415E5D4F7D
:103790004A01FA012081222329F06A946110C7CFDF
:1037A000712C2DC020912001F601E21BF10927FDAB
:1037B000F3959F01F7FF03C03195219531094091A1
:1037C0001F01C41BD10947FDD395D7FF03C0D19575
:1037D000C195D1092C0F243000F3C80ED91EF50174
:1037E000EC0DF11D80818F3FC1F27720B1F26E2D7B
:1037F000802F0E94631887FFD0CFF4015082872D5D
:10380000DF91CF911F910F91FF90EF90DF90CF90BC
:10381000BF90AF909F908F907F906F905F90089532
:103820002F923F924F925F926F927F928F929F92D0
:10383000AF92BF92CF92DF92EF92FF920F931F93BE
:10384000CF93DF93CDB7DEB7C058D1400FB6F89411
:10385000DEBF0FBECDBF611571058105910521F455
:1038600066E270E282E590ED6093040170930501D9
:10387000809306019093070160930001709301010A
:103880008093020190930301EFE1F2E081E08193E4
:1038900023E0EF31F207D9F710921E02109236039F
:1038A0001092370310923503109234038093200155
:1038B00080931F018093380310923002CF5FDE4F58
:1038C0008883C150D140CF5BDE4F8883C154D14043
:1038D00011E0F3E04F2EC12ED12CC6010197E1E09B
:1038E000F1E0EC0FFD1FE80FF91F6080A1E4B1E0EB
:1038F000AC0FBD1F8A0F9B1FFC0150801982F1E0A5
:10390000FA8322E02B834C82CE0101967C014C018C
:10391000B12CA12C782E0F2D63E070E0C5010E9420
:10392000271AD4019C91F701E80FF11D80818D9336
:103930004D019083BFEFAB1ABB0AE4E0AE16B104B1
:1039400059F75701F4E0AF0EB11CD7018D917D01FD
:1039500090E0FC01E95AFE4F2080322C330C360CEB
:10396000855A9E4FFC019080892C880C850C8FEF26
:10397000830D8E3008F070C08FEF880D8E3008F008
:103980006BC0682D832D0E94421A813009F064C0FB
:10399000590CF0E15F9EC0011124620C815E9D4FC5
:1039A000860D911DDC011C92B0E18B9EF00111246B
:1039B000E15EFD4FE30DF11D1082E1E0F1E0EC0F5F
:1039C000FD1FEC0DFD1D3082E1E4F1E0EC0FFD1F69
:1039D000EC0DFD1D80821F5F11117DCF6DE070E049
:1039E00084E090E00E94271AC82ED12CDC1408F045
:1039F00053C06DE070E082E090E00E94271A7C01E5
:103A00006DE070E082E090E00E94271ADC01BB27A5
:103A1000E4E0AA0FBB1FEA95E1F797013327F9010C
:103A2000EA0FFB1FE15EFD4F4081413099F5BD017A
:103A3000615E7D4F4FEF4E0D460F572F511DDA013E
:103A40004C9141110FC0E394DB01AE0DB11D4C91BF
:103A5000411108C010821EC0EA14FB0409F075CFA2
:103A60001150BACFAFEFA80F40E1A49FD0011124AD
:103A7000215E3D4FA20FB31F4C9141110BC08F5FD0
:103A8000A0E18A9FC0011124280F391FD9018C9110
:103A9000882301F3D394AACF872D902F0E94C21AB6
:103AA0007FE2A72E72E0B72E6E01B1E1CB0ED11CE2
:103AB000A601B501F0E021E1E1E181E090E0FF2421
:103AC000FA94F20EDB01A80FB91F3C9131110BC023
:103AD000DA01A80FB91F3C913F3F29F0F31718F402
:103AE000EF2DE80FF32F01968F30910559F7605FA6
:103AF0007F4F405F5F4F205F213FF9F6F0E0E15ECE
:103B0000FD4F82E08083872D902F0E94C21A9090F3
:103B10002101892D8370672D702F29F485E00E9483
:103B2000841B672D702F85E00E94841BF92CFF0CED
:103B3000F90CE7E0FE0EFEE0FF1510F46EE0F62E45
:103B4000E12C672D702FEF1429F084E00E94841B74
:103B5000E394F7CF86E00E94841B672D702F83E0EB
:103B60000E94841B81113CC0812C51E1752E01E023
:103B7000EE24E394F12C55245A94570CF501EE0DE4
:103B8000FF1D8081811112C0F601EE0DFF1D6080C6
:103B90002FEF621659F0861448F4602F8E2D0E9484
:103BA000631887FF03C0152D1E0D862C3FEFE31A07
:103BB000F30A4FE0E416F10409F70F5F80E1C80E45
:103BC000D11C90E1790EA0E1AA0EB11C0F3081F654
:103BD000882031F0E12FF0E0E15EFD4F83E080834B
:103BE00033E0C32EC90CB6E0BC1510F426E0C22E9B
:103BF000B92CB694B39411E0190DD0901E02DC14C8
:103C000008F05FC00AE56EE070E081E090E00E949D
:103C1000271A7C016EE070E081E090E00E94271A94
:103C200097013327AC015527FA0194E0EE0FFF1FEF
:103C30009A95E1F7E15EFD4FE20FF31F608161119C
:103C40003DC02150310937FF03C03195219531091D
:103C50004150510957FF03C0519541955109240F17
:103C6000263060F1F82EAE2C682F8E2D0E9463183E
:103C700087FF24C0612F173008F066E070E090E005
:103C800080E00E94271A082F63E670E090E080E051
:103C90000E94271A8D9714F40111015024E0D29E3E
:103CA000F0011124E35CFC4FA082F18203830695AE
:103CB0000B0D0283D394D0921E029FCF015009F0C6
:103CC000A2CF84EA91E00E947A18C058DE4F0FB666
:103CD000F894DEBF0FBECDBFDF91CF911F910F9142
:103CE000FF90EF90DF90CF90BF90AF909F908F901C
:103CF0007F906F905F904F903F902F900895EF923C
:103D0000FF920F931F93CF93DF93D82FC62F0E945C
:103D1000421A8130B1F40BE511E087E5E82E81E02D
:103D2000F82EF80161918F01F70181917F016C0FED
:103D30008D0F0E94421A813031F4F1E00F351F07D8
:103D400081F780E013C090910501809121012BE063
:103D5000829F900D112485E2D89F900D1124E7E1F8
:103D6000CE9F900D11249F7081E059F7DF91CF9184
:103D70001F910F91FF90EF9008950E94421A9FEFBC
:103D8000980F81E0923008F080E008952F923F92E2
:103D90004F925F926F927F928F929F92AF92BF925B
:103DA000CF92DF92EF92FF920F931F93CF93DF9307
:103DB000CDB7DEB763970FB6F894DEBF0FBECDBFA9
:103DC0000E94BA0D8091380390E09C012D5F3F4F17
:103DD00023703327F901E95AFE4F40814C83255A5D
:103DE0003E4FF901F081FD83019683709927FC0114
:103DF000E95AFE4F20812E83855A9E4FFC01F081A7
:103E0000FF8367E3662E61E0762E73E0572E809184
:103E1000380390E0FC01E95AFE4F208140902001D8
:103E2000529E400C1124855A9E4FFC018081F090D7
:103E30001F01589EF00C1124F9826F2D842D0E94D1
:103E4000421AE82EF1E08F1311C1F301268837885A
:103E500084889588A288B388C088D188E82C01E03E
:103E6000222D482DB501C6010E940C1200E0222D22
:103E7000482DB501C6010E942E123B822A8237FED0
:103E800005C091012D5F3F4F3B832A838A819B812F
:103E900095958795959587959B8B8A8B039724F4A9
:103EA000E3E0F0E0FB8BEA8BC40197FC03969C01F6
:103EB00035952795359527953B832A832530310500
:103EC00024F485E090E09B838A830A891B890A0D8C
:103ED0001B1DF101EA0DFB1DF987E887288539854F
:103EE000021713070CF43FC08A819B819595879533
:103EF0009D878C877501F401EC0DFD1DF98BE88B16
:103F00002A893B89235031093B872A87E885F9852F
:103F1000EE16FF06C4F5C7016A897B890E94413706
:103F20008B010170112760FF02C00C851D850C0DEF
:103F30001D1D97012E5F3F4F3F872E8788899989E6
:103F400008171907DCF4EA85FB85EF2B39F020E030
:103F50004A856E857F85C8010E94E3112A813B81D5
:103F6000020F131FEBCF20E04E2DB801C6010E94B7
:103F7000DD0D8A899B89080F191FB0CF8A899B891B
:103F8000E80EF91EC3CF6981842D0E947F1EE82EA2
:103F9000882309F44CC06D819981690F8C81840D4F
:103FA0000E94421A8130D1F46F81E9816E0F8E81B7
:103FB000840D0E94421AE12C813081F4F9818F2F07
:103FC000FF0F990B840D911D47FC9A95E0902101FC
:103FD000E80EF92EF11C2E2D2170E22E37FE03C0C3
:103FE0003FEF231A330A35942794222D2D3108F000
:103FF0002CE1203108F420E1422F46952A0C3B1C8D
:10400000B101640F711D8091550300EE15E084FD30
:1040100002C000ED15E097FE03C08FEF881A980AE2
:1040200095948794C4018C0D9D1D0E94990F48E0C2
:10403000641A71085A945110EACE63960FB6F89438
:10404000DEBF0FBECDBFDF91CF911F910F91FF90CB
:10405000EF90DF90CF90BF90AF909F908F907F9028
:104060006F905F904F903F902F90089592E089134A
:104070008AC081E080933503F3014688378824891C
:1040800035893B832A83C288D388E088F18801E0A0
:10409000242D4A81B601C7010E940C1200E0242D94
:1040A0004A81B601C7010E942E122CEF240D4A81CD
:1040B0004650B6016E5F7F4FC70103960E942E12D5
:1040C0008701085F1F4FAA80BB80AE0CBF1C34E085
:1040D000A31AB1088AEF282E240C460143E0840E6F
:1040E000911C0A151B054CF420E0422DB401C801B7
:1040F0000E94E311075F1F4FF4CF8A819B8167E025
:1041000070E00E944137242D332D37FF02C0295F14
:104110003F4F03E0359527950A95E1F7AB016330F2
:10412000710514F443E050E02230310514F422E02C
:1041300030E0642D732D77FF02C06F5F7F4F759560
:1041400067956C0D7D1DC90137FD01969595879585
:10415000681B790B8A819B8197FF03C001969B8323
:104160008A83EA81FB81F595E795CF018E0D9F1D2E
:10417000FA0157FD3196F595E79500E08E1B9F0BF0
:104180000E940C1254CFF6E08F1303C081E080939D
:1041900034039301205F3F4F3B832A838301085EF2
:1041A0001F4FCD803981C30EDC80D40C6C2D8D2D3A
:1041B0000E94BD1E882391F040E0B8018A819B8156
:1041C0000E9435166C2D8D2D0E947F1E882331F0A4
:1041D00040E0B8018A819B810E945514CF804981BB
:1041E000C40EDE80D40C6C2D8D2D0E94BD1E882344
:1041F00091F041E0B8018A819B810E9435166C2DB7
:104200008D2D0E947F1E882331F041E0B8018A8104
:104210009B810E9455146981842D0E94631887FD3B
:104220001BC094E08902F0011124E35CFC4F838100
:10423000873008F086E090E0FC01EF57FC4E449197
:10424000FC01EE0FFF1FE857FC4E6591749123E7C8
:10425000852D0E94F515EBCEE3E04BE460E976E0B6
:10426000EE1631F0F4E0EF1207C041E460E776E0CB
:10427000852D0E946F13DBCE25E0E2120BC08091EA
:10428000550360E576E084FD02C060E376E02BE450
:1042900040E1DECF36E0E312CACE8091550360E103
:1042A00076E084FD02C060EF75E025E5F1CFCF92A6
:1042B000DF92EF92FF920F931F93CF93DF93C09003
:1042C0001E02E0902001D0901F01CDE3D3E0F12C3D
:1042D000CF1409F450C08A8118160CF043C008812D
:1042E0005E2D501B19814D2D411B252F052E000CD5
:1042F000330B37FF03C0319521953109842F042EEC
:10430000000C990B97FF03C0919581959109622F3D
:10431000680F623058F48F2DDF91CF911F910F916C
:10432000FF90EF90DF90CF900C94FE196730D0F49F
:1043300082179307D4F48FEF15160CF481E0080F61
:10434000612F802F0E94BD1E81110CC0612F802F14
:104350000E94631887FF06C0E01202C0D11611F058
:1043600008831983F3942496B3CF8FEF14160CF4BB
:1043700081E0180FE5CFDF91CF911F910F91FF9052
:10438000EF90DF90CF900895FF920F931F93CF93FC
:10439000DF93F82E8091380390E0FC01E95AFE4F3C
:1043A000D08120912001D20F855A9E4FFC01C081FF
:1043B00080911F01C80F6C2F8D2F0E94631887FDFD
:1043C00007C0DF91CF911F910F91FF900C94FE19C0
:1043D0006C2F8D2F0E94BD1E81112DC08F2D90E05E
:1043E000FC01E95AFE4F10811D0F855A9E4FFC01BA
:1043F00000810C0F602F812F0E94421A8130D9F06A
:10440000D0932001C0931F01F09238030E949D18A1
:104410000E94541A80916C03833079F4602F812FAD
:104420000E94631887FFCDCFDF91CF911F910F912D
:10443000FF900C945721F0923803DF91CF911F9198
:104440000F91FF900895CF93DF93D0912001D80F63
:10445000C0911F01C60F6C2F8D2F0E94631887FD1E
:1044600004C0DF91CF910C94FE196C2F8D2F0E9408
:10447000421A823079F58091360381110BC08CEAA3
:1044800091E00E947A1866E08EE690E0DF91CF918D
:104490000C947919C0912101CF5FC093210129E1CA
:1044A000C29FC00111248C599F4F0E94B3180E94D3
:1044B000C2198C270E94101C83EB91E00E947A188D
:1044C00025E048EB51E064E084E992E0DF91CF9190
:1044D0000C94E2186C2F8D2F0E94BD1E811110C00C
:1044E000D0932001C0931F010E949D180E94541A6E
:1044F00080916C03833051F4DF91CF910C9457215C
:1045000088EB91E0DF91CF910C947A18DF91CF91F5
:104510000895089590E080E008958F929F92AF9261
:10452000BF920F931F93CF93DF93CDB7DEB7A197C1
:104530000FB6F894DEBF0FBECDBF19A2423008F40B
:104540004AE08E010F5D1F4F842E912CB12CA12CBF
:10455000A50194010E94D734E62FB901CA01EA30BF
:1045600044F5E05DD801EE938D01232B242B252B00
:1045700079F790E080E0109769F0FD01019000204C
:10458000E9F73197AF014A1B5B0BBD018CED97E05A
:104590000E94780DA1960FB6F894DEBF0FBECDBF76
:1045A000DF91CF911F910F91BF90AF909F908F900F
:1045B0000895E95CD7CF0F9300E029E040E867E376
:1045C00070E090E080E00E940C1282E090E0909316
:1045D00063038093620388E390E090936103809388
:1045E000600348E051E0FA0101900020E9F7AF01D3
:1045F0004950514068E071E08CED97E00F910C94C8
:10460000780D8F929F92AF92BF92CF92DF92FF92DE
:104610000F931F93CF93DF9300E029E040E867E317
:1046200070E090E080E00E940C1281E090E09093B6
:1046300063038093620388E390E090936103809327
:10464000600386EB96E00E94C81100911E0110E005
:104650002091220130E044E169E388E00E942613C2
:10466000F0906803D091690300916A0310916B0385
:104670002F2D3D2FA801C1E06AE0862E912CA12CA0
:10468000B12C2A3031054105510540F0CA01B9016C
:10469000A50194010E94D734CF5FF3CF23E02C0F04
:1046A0003AEF3203C001112480589F4F97FD0196C5
:1046B00095958795082E000C990B90936303809332
:1046C000620338E3C32ED12CD0926103C092600301
:1046D00080EB96E00E94C8114AE06F2D7D2FC80143
:1046E0000E948D2288E690E090936303809362039A
:1046F000D0926103C092600384EB96E00E94C811DF
:104700000E94911820915C0330915D038C0140E17F
:1047100069E38FE60E942613DF91CF911F910F91DD
:10472000FF90DF90CF90BF90AF909F908F900895B3
:10473000682F70E090E080E04AE00C948D22AF9208
:10474000BF92CF92DF92EF92FF920F931F93CF937E
:10475000DF9300E028E040E870E060E090E080E077
:104760000E940C1281E0809327018093280181E050
:1047700090E0909363038093620310926103109220
:10478000600380EE96E00E94C8110091350110E0B0
:104790002091360130E042E162E08EE00E94261373
:1047A00085E290E09093630380936203109261032B
:1047B000109260038EED96E00E94C8118091210155
:1047C0000E94982387E390E09093630380936203B1
:1047D000109261031092600380913603882309F4DC
:1047E000CBC088ED96E00E94C81181E590E09093DF
:1047F00063038093620310926103109260038CED57
:1048000096E00E94C811609158037091590390E09E
:1048100080E04AE00E948D2288E790E09093630355
:1048200080936203109261031092600380913803B9
:104830008111A5C082ED96E00E94C8110E9401235B
:1048400080913B0381110E94DB22809137038823F2
:1048500009F451C100E02BE248E36AE070E081E036
:1048600090E00E940C1201E02BE248E36AE070E065
:1048700081E090E00E942E1281E0809327018093D6
:104880002801C4E0D0E0D0936303C09362038DE0BD
:1048900090E0909361038093600387EC96E00E9420
:1048A000C811809125010E949823D0936303C0937F
:1048B000620387E190E0909361038093600382EC50
:1048C00096E00E94C81180915B030E949823D093C8
:1048D0006303C093620381E290E09093610380934D
:1048E00060038EEB96E00E94C811809136010E9411
:1048F00098238CEB96E00E94C811809135010E94AC
:104900009823D0936303C09362038BE290E090936B
:1049100061038093600388EB96E00E94C811809148
:1049200026010E94982300E022E342E369E070E060
:104930008DE490E00E940C1201E022E342E369E082
:1049400070E08DE490E00E942E129FE1C92E92E06B
:10495000D92ECAE0D0E056018EE4E82EF12CF50104
:1049600081915F018130C1F401E023E043E0BE01A9
:10497000C7010E940C1222C084ED96E034CF813032
:1049800019F480ED96E058CF823019F48EEC96E061
:1049900053CF8CEC96E050CF823009F03EC080912E
:1049A0003503882359F08091550384FF07C001E047
:1049B00023E043E0BE01C7010E942E12F3E0EF0E98
:1049C000F11C8EE7E816F10451F6239690E1C90E2A
:1049D000D11CCA33D10509F0BECFC0E0D3E080912D
:1049E0001E02C81728F584E0C89FF0011124E35C7B
:1049F000FC4F828118167CF461816D02B001112494
:104A0000655F7F4F80818D02C001112441E0815B91
:104A10009F4F0E947B0FCF5FE2CF863079F6809167
:104A20003403882359F28091550384FFC7CF9CCF6C
:104A3000C0901F018C2D880F8C0D865FC82ED12C45
:104A400080912001C82FCC0FC80FC25BD0E0B60107
:104A50006150710900E025E045E0CE0101970E9418
:104A60000C128091380376019FEFE91AF90A8E0142
:104A70000F5F1F4F41E0B6018823E9F05601E2E0E5
:104A8000AE0EB11C41E0813099F4B701CE0102961F
:104A90000E947B0F41E0B601C8010E947B0F41E0FC
:104AA000B701C8010E947B0F41E0B501C80114C0E5
:104AB0008230F1F4B501C8010E947B0F41E0B701DB
:104AC000CE010E947B0F41E0B701C8010E947B0F1D
:104AD00041E0B701CE010296DF91CF911F910F9176
:104AE000FF90EF90DF90CF90BF90AF900C947B0F32
:104AF000B701CE01CDCFDF91CF911F910F91FF90E4
:104B0000EF90DF90CF90BF90AF9008950C946334F6
:104B100082E090E00E94862581110C94B70D0C94E0
:104B2000B40D1F920F920FB60F9211248F939F9383
:104B30008091E1009091E100937F9093E10083FFE9
:104B40000FC01092E90091E09093EB001092EC00FE
:104B500092E39093ED0010928B0398E09093F00015
:104B600082FF22C093E09093E9009091F200992394
:104B700019F09AE39093E80090917C03992341F017
:104B800090917C03915090937C03911101C05D9AA8
:104B900090918A03992341F090918A0391509093C8
:104BA0008A03911101C0289A84FF18C08091E20005
:104BB0008E7E81608093E2008091E1008F7E809301
:104BC000E10080917D038E7E806180937D039F91C3
:104BD0008F910F900FBE0F901F90189580FFF7CF09
:104BE0008091E2008E7E80618093E2008091E100FE
:104BF0008E7E8093E10080917D038E7E8160E5CF83
:104C00001F920F920FB60F921124CF92DF92EF9264
:104C1000FF920F931F932F933F934F935F936F9345
:104C20007F938F939F93AF93BF93EF93FF93CF9314
:104C3000DF93CDB7DEB76C97DEBFCDBF1092E90032
:104C40008091E80083FF25C068E0CE0145960E9470
:104C50008E0C82EF8093E8008D8987FF39C0909198
:104C6000E80090FFFCCF982F907609F034C19E8920
:104C70004F89588D2F89F88C911131C0803861F59A
:104C800080917B038093F1001092F1008EEF80936E
:104C9000E8006C960FB6F894DEBF0FBECDBFDF9173
:104CA000CF91FF91EF91BF91AF919F918F917F91A4
:104CB0006F915F914F913F912F911F910F91FF90B5
:104CC000EF90DF90CF900F900FBE0F901F90189530
:104CD0009EEF9093E800C7CF1092F100D5CF9130AE
:104CE00059F48111D3CF4130510581F680917B0376
:104CF0008D7F80937B03CACF933049F48111C6CF57
:104D00004130510519F680917B038260F2CF9530D6
:104D100041F48091E80080FFFCCF20682093E300FD
:104D2000B5CF963009F0A9C00B8D1C8D22E01092F2
:104D3000E9001092790310927803F2122EC01092BB
:104D40007703109276030E945D0C1F8299E099838D
:104D5000FA8291E09E8390EA98879AEF9987209152
:104D6000780330917903275F3F4F3C832B838D83FA
:104D70001092E90010927903109278031093770350
:104D80000093760349E050E0BE016F5F7F4F80E003
:104D90000E94370C0E945D0C79CF1093770300932B
:104DA00076030E94740BDC0112960D911C91011583
:104DB000110509F451C1D801ED91FC910480F581F0
:104DC000E02DBE016B5E7F4FC8010995009709F089
:104DD0003EC1F80100851185EACFF3E0FF120EC055
:104DE0008F89882309F440C0823061F440E860E193
:104DF0008FE594E10E947C28811148CF81E2809365
:104E0000EB0047CF813029F440E86BE083E594E183
:104E1000F1CF833099F70E94740BDC011296ED906C
:104E2000FC908E010F5F1F4F6801E114F10479F0CF
:104E3000D701ED91FC910680F781E02DB801C70103
:104E40000995080F111DF701E084F184EECFD80118
:104E50001C92F60101900020E9F73197BF016C190F
:104E60007D0940E0C601C6CF6DE374E1FB014491CA
:104E700050E080E80E94370C09CF973009F4BECF8C
:104E8000983021F481E08093F10000CF993009F04F
:104E9000FDCE837009F0B2CFE0E6F1E081E031E0D1
:104EA00096E32191222371F08093E9003093EB0087
:104EB000DF0111972C912093EC009093ED008F5F10
:104EC000873079F78EE78093EA001092EA008F89A5
:104ED00080938B03DBCE8B8D9C8D1092E90010921A
:104EE0007903109278039093770380937603898DEA
:104EF000811192C08E899D89913A49F4813209F0DD
:104F00007DCF47E050E06DE271E080E0B3CF9132B9
:104F100009F074CF833269F48F89988DB0E0A0E0F6
:104F20008093290190932A01A0932B01B0932C0127
:104F3000ADCE803269F48091E80082FFFCCF67E05B
:104F40008DE291E00E948E0C8BEF8093E8009ECE64
:104F5000823209F09BCE8F8980933401EEEFFFE718
:104F6000859194918B3F9C4D51F1E0E0F8E0809168
:104F70002D0190912E01A0912F01B0913001803B25
:104F80009440A105B105F1F48091340180FD1AC06F
:104F9000EE3F8AE0F80789F587E797E791838083FA
:104FA0008091600080937A0388E19BE00FB6F894CB
:104FB000A895809360000FBE9093600067CEEEEFDF
:104FC000FAE0D5CF808191818737974709F05ECE8F
:104FD000A8958091600088618093600080917A0339
:104FE00080936000EE3F2AE0F20789F08091FE0A8C
:104FF0009091FF0A9183808349CE80819181873788
:10500000980751F29093FF0A8093FE0AC5CF109241
:10501000FF0A1092FE0A3ACE0E94740BDC0112962F
:105020000D911C910115110509F4E8CED801ED91FF
:10503000FC910190F081E02DBE016B5E7F4FC801B5
:105040000995811123CEF80100851185EBCF181643
:1050500019060CF41BCED2CEF1E0FF12BECE61E4F5
:1050600074E104CF1F920F920FB60F9211242F9369
:105070003F938F939F93AF93BF9380916E039091D3
:105080006F03A0917003B091710330916D0323E021
:10509000230F2D3758F50196A11DB11D20936D03E7
:1050A00080936E0390936F03A0937003B09371038A
:1050B0008091720390917303A0917403B091750372
:1050C0000196A11DB11D8093720390937303A09369
:1050D0007403B0937503BF91AF919F918F913F91EE
:1050E0002F910F900FBE0F901F90189526E8230F59
:1050F0000296A11DB11DD2CFEF92FF920F931F9385
:10510000CF93DF93F82E192FE62E042F81E0860F20
:10511000880F0E94090C83E00E94090CCF2DD12F2B
:10512000EC0EFD2EF11CCE15DF05B9F007FF13C004
:10513000FE0184910E94090C182F80E00E94090C46
:10514000812321968111EFCFDF91CF911F910F9194
:10515000FF90EF9008958881EDCF81E0F5CFECE8E6
:10516000F7E01382128288EE93E0A0E0B0E084833F
:105170009583A683B7838AE691E0918380838FEF3E
:105180009FEF95878487ECEDF7E0138212828CE71E
:1051900091E0918380830895789484B5826084BD82
:1051A00084B5816084BD85B5826085BD85B581602B
:1051B00085BD80916E00816080936E0010928100A9
:1051C0008091810082608093810080918100816064
:1051D0008093810080918000816080938000809125
:1051E0009100826080939100809191008160809312
:1051F0009100809190008160809390008091C10027
:1052000084608093C1008091C10082608093C1005E
:105210008091C10081608093C1008091C300816052
:105220008093C3008091C00082608093C000809111
:10523000C20081608093C20080917A008460809374
:105240007A0080917A00826080937A0080917A005F
:10525000816080937A0080917A00806880937A00E0
:1052600010928B0310927B0310927D038091D700E4
:1052700081608093D70080EA8093D80089B58061EF
:1052800089BD89B5826089BD09B400FEFDCF61E0AA
:1052900070E080E090E00E94C00C8091D8008F7C8C
:1052A00080618093D8008091E000807F8093E0004F
:1052B0008091E1008E7E8093E1008DE08093E2009A
:1052C000559A209A81EC80937C0085B1806F85B9D6
:1052D00084B1877E84B984B1876E84B95E9A5F9801
:1052E0008AB1806D8AB9769A6E9881B3806F81BBDE
:1052F000899880B38D7080BB80E58CBD81E08DBDC9
:1053000085E090E00E94A70D5F9A85E090E00E9402
:10531000A70D5E985C98E5E9FCE082EA9CE02491A8
:105320002EBD00000DB407FEFDCF31968E179F07EE
:10533000B1F75C9A81E88093640080916500816098
:10534000809365000E94DA0D0E94AC0D87FF15C0A6
:105350005C9885EA8EBD00000DB407FEFDCF5C9A17
:105360002E982F982D98809164008062809364001D
:1053700081E083BF889513BEFCCF0E94AC0D82FFF5
:1053800048C02D980E94AC0D84788438E1F40E94C6
:10539000A50D88EC90E00E94A70D2F9882E090E088
:1053A0000E9463348F3F29F06FEF82E090E00E940B
:1053B0007D3484EF91E00E94A70D2F9A0E94AC0DDE
:1053C00084788438D9F30E94AC0D84718431E1F47F
:1053D0000E94A50D88EC90E00E94A70D2E9882E017
:1053E00090E00E946334882329F060E082E090E03E
:1053F0000E947D3484EF91E00E94A70D2E9A0E94B6
:10540000AC0D84718431D9F388EC90E00E94A70D33
:10541000B4CF0E94A50D0E94882581E090E00E94F3
:105420008625182F147081FF0CC011112E98C1EF22
:10543000DFEF0E94AC0D86FF5DC02E9A2F9A0E946E
:10544000A50D82E390E00E94A70D0E94AC0D811192
:10545000F8CF81E280931A010E9488251092900073
:105460008AE0809391001092C00088E08093C10090
:105470001092C3001092BF001092CF000E94B40D92
:1054800080E190E00E946B34609364037093650345
:1054900080936603909367036F3F7F4F8F4F9F4FBB
:1054A00041F4109264031092650310926603109207
:1054B0006703C4E14C2E512C612C712CB6E22B2ECB
:1054C000312C2FB7F89480916E0390916F03A091C7
:1054D0007003B09171032FBF20912103222309F49F
:1054E00061C01092210380E090E0892B51F30E946B
:1054F0000000E4CF112329F0C430D10511F42E9A15
:105500002F9881E00E942A0B00E128E545EE5BE040
:10551000BE0184E190E00E946F0A0E94DA0D8FE0E4
:1055200090E00E94A70D2196C931D10509F081CFE5
:10553000112311F02F9A2D9880E991E00E94A70D78
:105540000E94A50D81E090E00E94862580FF79CF22
:105550008AE090E00E9486259FEF980F9E3F08F01A
:1055600070CF22E330E0309363032093620328E39B
:1055700030E03093610320936003CBE0D0E0682FEC
:105580008CED97E00E941511CE010E948625219690
:10559000C131D105A1F70E94DA0D88EE93E00E9497
:1055A000A70D4FCF20912203382F321B232F30918C
:1055B0001A01231748F42F5F231708F094CF81E0D6
:1055C00083BF889513BE8FCF21E020932103809362
:1055D000220380911F039091200301969093200352
:1055E00080931F0380912A03882339F08150809390
:1055F0002A03811102C01092900080912903882310
:1056000039F0815080932903811102C01092C000AB
:10561000809126038823C9F181508093260381114C
:1056200034C060912403709125036115710569F1FF
:1056300080913103882329F190E080E00E941636A2
:105640006B017C0120E030E040E05FE30E94A43683
:1056500020E034E244E759E40E940935A7019601AD
:105660000E9475350E94E7356150710980912303CE
:1056700080932A0380E48093900070939900609354
:1056800098001092250310922403809128038093A0
:1056900027030E94AC0D8093280380916C03811135
:1056A00027C080911B01882319F0815080931B0132
:1056B00080911B01882351F088E00E94CF0D811159
:1056C00005C084E00E94CF0D882319F081E080930B
:1056D0006C030E94BA0D00E420E842EA5CE070E04E
:1056E00060E090E080E00E946F0A0E94DA0DFBCE3D
:1056F000813009F000C2809155038F5F809355037C
:1057000080E80E94CF0D811105C080E10E94CF0D7D
:10571000882331F08091320391E08927809332030E
:1057200084E00E94CF0D81110E94AD1988E00E9493
:10573000CF0D882359F080913203811112C00E944D
:10574000C81810925F0382E080936C03809131034C
:10575000882321F080916C03813031F00E94C818B9
:1057600021C00E94AD19F2CF8FB7F894C0906E039C
:10577000D0906F03E0907003F09071038FBF809121
:105780002D0390912E03A0912F03B0913003009729
:10579000A105B10509F4D7C0C816D906EA06FB066B
:1057A00008F0D1C00E94BA0DC0E010E000E0D3E1E3
:1057B00062E2862E912C2091550330E08C2F63E01D
:1057C0000E942137492F50E04F5F5F4F429FC00139
:1057D000439F900D529F900D1124800F911FB40193
:1057E0000E9441377C015C019FEFA91AB90A3595E7
:1057F0002795CD9F200D11242F77822F90E06C01EB
:10580000EFEFCE1ADE0A41E0C0FF6CC1B7010E9483
:105810007B0F41E0B501C6010E947B0FCF5FDD5FCA
:10582000095F1F4FCE3039F601E02CE140E767E019
:1058300070E088E090E00E942E120AE120E742EA40
:1058400050E168E070E088E090E00E946F0A1091FB
:10585000320311110EC08FE190E0909363038093A7
:105860006203309261032092600382E692E10E941B
:10587000C811CBE2D0E0D0936303C09362033092AF
:105880006103209260038AE792E10E94C811D093DD
:105890006303C09362038FE290E09093610380936F
:1058A000600383E792E10E94C8118091310388234D
:1058B00009F41EC180E792E10E94C811113081F401
:1058C0008FE190E090936303809362038FE290E016
:1058D00090936103809360038AE692E10E94C8116D
:1058E00081E290E0909363038093620388E390E009
:1058F000909361038093600384E692E10E94C81153
:1059000060916403709165038091660390916703D1
:105910004AE00E948D22E9CE2FEFAC0140395105BB
:1059200008F0DBC0CA010196FA01EA54FD4EC491A9
:10593000C03F91F490932C0380932B0320931D017F
:1059400030931C010BCF30911C0140912B035091DF
:105950002C0320911D01E2CF70E77C0F723078F4A8
:1059600080399105D1F24E5F5F4FFC01EA54FD4E44
:10597000C03919F42491CA01D0CF3491FCCF70E81A
:105980007C0F723028F4C03809F4C6CF3FEFC5CF82
:1059900090932C0380932B0320931D0130931C01C3
:1059A0008039910509F4DACE4E5F5F4F50932C0396
:1059B00040932B03FC01EA54FD4EE491DC2FCE2FE3
:1059C00027FF02C037FD7CC0CE0161E270E00E947B
:1059D0002D37162F6F3008F01EE0123008F412E059
:1059E00027FD36C089EC820F8B3168F4822F8753F4
:1059F000990BFC01EE0FFF1FE058FD4E659174916D
:105A00006115710511F468EB71E090E080E00E948F
:105A100016364B015C0120E030E040E05FE30E947D
:105A2000A43620E034E244E759E40E940935A50198
:105A300094010E9475350E94E735615071091093F9
:105A40002A0380E4809390007093990060939800FB
:105A5000E0911C01E7FD34C089EC8E0F8B3158F4C6
:105A6000E753FF0BEE0FFF1FE058FD4E6591749159
:105A70006115710511F468EB71E090E080E00E941F
:105A800016364B015C0120E030E040E05FE30E940D
:105A9000A43620E034E244E757E40E940935A5012A
:105AA00094010E9475350E94E73561507109109389
:105AB000290380E48093C0007093BF006093D100FD
:105AC000CC0EDD1EE11CF11CC0922D03D0922E03E2
:105AD000E0922F03F092300365CE50932C03409355
:105AE0002B032CCFB5010E947B0F41E0B70193CE71
:105AF0008CE692E1E1CE823009F02BC180E20E9477
:105B0000CF0D882359F080915F038D5F8370809360
:105B10005F0362E08CEB92E00E94791980E40E94BE
:105B2000CF0D882359F080915F038F5F837080933E
:105B30005F0362E08CEB92E00E94791984E00E949E
:105B4000CF0D882309F485C063E080EF90E00E94C8
:105B5000791981E080936C030E94BA0D81E08093F3
:105B600027018093280189E190E09093630380935B
:105B7000620322E030E030936103209360038BE7FF
:105B800093E10E94C811F12CC2E1D0E033E020E1A2
:105B9000F31222E14CE150E0BE018F2D0E94AE15C0
:105BA00010915F031F1109C001E026E146E169E0A1
:105BB00070E0CE010B970E942E12F3946F9684E052
:105BC000F812E4CF3092630320926203E3E2F0E044
:105BD000F0936103E093600383E593E1112351F0B7
:105BE0008FE493E1113031F08BE493E1123011F046
:105BF00086E493E10E94C8118CE190E090936303E6
:105C0000809362038DE290E0909361038093600340
:105C100084E793E1112351F08CE693E1113031F0E8
:105C200084E693E1123011F08FE593E10E94C811F0
:105C300084E190E0909363038093620388E390E0B3
:105C4000909361038093600388E593E10E94C811FB
:105C50004CCD88E00E94CF0D882309F47DCFC09100
:105C60005F0322E04CED55E062E088EE93E00E9495
:105C7000E218C093230181E080932101109259031F
:105C8000109258038093260110925D0310925C03DA
:105C9000109268031092690310926A0310926B03CA
:105CA000109236031092370310923503109234038A
:105CB00010923303C11131C098E090933501809365
:105CC000250110925B0390931E0180913501809312
:105CD000360180911E01809322010E94C2194B015E
:105CE0005C018FB7F894C0906E03D0906F03E09082
:105CF0007003F09071038FBF0E949B0C7601DD242E
:105D0000CC24682579258A259B256C257D258E2523
:105D10009F250E94101C83E01DCFC13059F486E0FE
:105D20008093350194E09093250110925B0380935A
:105D30001E01CBCF96E09093350180932501C230B0
:105D400021F484E080935B03BECF10925B0384E078
:105D5000EECF833009F089C0809155038F5F809327
:105D6000550380913B03882319F0815080933B03B6
:105D700080E20E94CF0D882331F0809138038D5F3F
:105D800083700E94C42180E40E94CF0D882331F0EB
:105D9000809138038F5F83700E94C42180E80E9445
:105DA000CF0D882369F08091380390E0FC01E55A1B
:105DB000FE4F895A9E4F6081FC0180810E94232200
:105DC00080E10E94CF0D882379F08091380390E024
:105DD000FC01E55AFE4F60816195895A9E4FFC0196
:105DE000808181950E94232288E00E94CF0D882324
:105DF00011F18091380390E0FC01E95AFE4FC08117
:105E0000855A9E4FFC01D08160911F016D0F8091DA
:105E100020018C0F0E94421A863011F510925A030D
:105E200085E080936C0323E04CE454E062E080E280
:105E300093E00E94E21884E00E94CF0D882359F07D
:105E40008091370391E089278093370362E088E5EA
:105E500092E00E9479190E94C61E0E949F2345CCA1
:105E60006D2F8C2F0E942322E6CF843009F01CC3B3
:105E7000809155038F5F8093550380913B03882366
:105E800019F0815080933B03D0915703DD2309F42F
:105E9000DDC0D150D0935703D11140C080913A0357
:105EA000882309F45FC0E0912401E7FD5BC01092F4
:105EB0003A0324E0E202F0011124E35CFC4FC381C9
:105EC0001282809158039091590301962C2F2695A8
:105ED000820F911D90935903809358033AE0C39F1A
:105EE000C001112449960E94B3188FEF80932401BA
:105EF00083E080936C0381E08C0F880F0E9452191D
:105F0000109239038DEB91E00E947A1824E048EE5C
:105F100053E063E084E992E00E94E2180E94C61E0A
:105F200000E028E340E868E070E090E080E00E9454
:105F30000C120E9401231091240117FDD6CBD091A1
:105F40005703DD2309F4BCC4909156038091550397
:105F5000963009F0B3C481FFB3C46EEF82FDB1C4C3
:105F600062E0AFC4809139038823C1F210923903F3
:105F7000F090560386E080935603E0912401E7FDFC
:105F800022C084E0E802F0011124E35CFC4F82812E
:105F90001816CCF4C3810091210110915B030E947B
:105FA000C219A30192010E94D734611119C083EC78
:105FB00091E00E947A1823E04CE454E062E080E231
:105FC00093E00E94E21880916C03843009F0A6CF20
:105FD00096E0F91609F4A2CF8FE0809357039ECF85
:105FE0009BEA099F812D1124869501E0080FC99F26
:105FF000812D11248695800F199F112D112416953E
:106000006231E0F090E0880F991F01968F3F910573
:1060100019F010F08FEF90E0181710F4D82FD11B63
:106020008D2F0E94261989EC91E00E947A1827E0B2
:1060300042E350E066E086E490E0C3CF181710F426
:10604000D82FD11B8D2F0E942619BDCFC0912401BE
:10605000C7FD0AC0E4E0CE02E0011124FE01E35CCA
:10606000FC4F8281181624F083E080936C0356CF96
:1060700080E80E94CF0D81110FC080E10E94CF0DFA
:1060800081110AC080E20E94CF0D811105C080E419
:106090000E94CF0D882359F080913C0391E089271D
:1060A00080933C0362E08CEB92E00E94791988E0D7
:1060B0000E94CF0D882309F431CF00913C0382E088
:1060C000013009F081E010912501809356030130E1
:1060D00009F065C080912301833051F48EEC91E08A
:1060E0000E947A1864E08EE690E00E94791916CF3B
:1060F00023E0813021F025E0823009F424E0909102
:106100002201921718F485ED91E0EACF921B90934B
:106110002201811123C01C5F83E0809356038BED25
:1061200091E00E947A180E94C219A30192010E9474
:10613000D734C62F611136C081EF91E00E947A18E2
:10614000C1E0C09356038FE08093570364E088EC6E
:1061500090E00E947919C0933903E0CE823039F47F
:106160001D5F84E08093560381EE91E0DACF85E0F5
:106170008093560380915803909159030296C35C13
:10618000DC4F2B81820F911D90935903809358030C
:106190008AE090E00E94B31887EE91E0C2CF8DEEC6
:1061A00091E0BFCF6231B8F0812F90E0880F991F46
:1061B0008F3F910519F010F08FEF90E0182F87EFC7
:1061C00091E00E947A1824E044E155E063E084E81D
:1061D00093E00E94E218E091240124E0E202F00141
:1061E0001124E35CFC4F8281811B82839FE09093AA
:1061F0005703181624F081E080933A038FCEC23102
:1062000050F4013061F424E048E151E063E088E0BB
:1062100092E00E94E21881E0809339037FCE23E070
:1062200044EB50E063E08CE291E0F3CF60E0CEEF2E
:1062300082FFC2E0062E000C770B6A5E7F4F28E1DA
:1062400047E350E0809123010E94AE1534E0130231
:10625000F0011124E35CFC4F2381273008F026E095
:1062600030E0F901EF57FC4E0491F901EE0FFF1FEA
:10627000E857FC4E259134918C2FCC0F990B4CE1B3
:1062800063E270E08E599F4F0E94C114DD23D1F06C
:106290008091560301E0813009F093C028E130E09D
:1062A00044E550E066E270E087E290E00E945C1214
:1062B00029E130E045E550E067E270E088E290E0F7
:1062C0000E945C1281E0809327018093280182E084
:1062D00090E09093630380936203E9E0F0E0F09331
:1062E0006103E093600384EA93E10E94C811809106
:1062F00036010E94982382EA93E10E94C81180919E
:1063000035010E9498232CE330E0309363032093FF
:10631000620389E090E090936103809360038EE9CB
:1063200093E10E94C811E091240194E0E902F00198
:106330001124E35CFC4F628167FD60E0062E000CD7
:10634000770B880B990B4AE00E948D2280913B03CA
:1063500081110E94DB22C0913C0301E0C11100E0E9
:106360002AE04DE16BE270E08EE290E00E942E1296
:1063700001E0C13009F000E02AE04DE16BE270E09D
:1063800082E590E00E942E12E4E3F0E0F0936303D4
:10639000E0936203CDE2D0E0D0936103C093600349
:1063A0008AE993E10E94C81188E590E09093630325
:1063B00080936203D0936103C093600386E993E105
:1063C00045CC8330C9F42FE04FE064E170E083E412
:1063D00090E00E942E1229E049E062E170E088E539
:1063E00090E00E942E1226E130E046E550E063E2A4
:1063F00070E08CE290E064CF8430E9F424E130E096
:1064000040E650E06BE270E082E290E00E945C12B5
:1064100025E130E041E650E06CE270E083E290E09C
:106420000E945C1228E230E043E450E06FE170E04B
:1064300089E390E045CF8530C9F426E046E068E185
:1064400070E082E490E00E942E1224E044E066E1D5
:1064500070E08AE490E00E942E122AE230E04DE2E1
:1064600050E06DE170E089E590E02ACF863099F444
:106470002CE230E046E250E06FE170E084E590E02D
:106480000E945C122DE230E045E250E060E270E0F4
:1064900083E590E015CF2AE130E043E550E066E285
:1064A00070E08BE290E00CCF853009F0E4C080E82A
:1064B0000E94CF0D811105C080E20E94CF0D88237C
:1064C00059F080915A038D5F837080935A0362E084
:1064D0008CEB92E00E94791980E10E94CF0D81112E
:1064E00005C080E40E94CF0D882359F080915A03A3
:1064F0008F5F837080935A0362E08CEB92E00E947E
:10650000791984E00E94CF0D882309F450C063E01C
:1065100080EF90E00E94791983E080936C030E94E1
:10652000C61E0E949F2300E020E344E76AE070E07B
:1065300086E090E00E940C1201E020E344E76AE06C
:1065400070E086E090E00E942E1281E080932701A7
:106550008093280130926303209262032DE030E0A3
:10656000309361032093600384EC93E10E94C8118F
:10657000C0915A032C2F40E06DEB73E188E10E943B
:10658000F8122C2F41E066EB73E181E20E94F812D1
:106590002C2F42E06FEA73E18AE20E94F8122C2F5E
:1065A00043E068EA73E183E30E94F8129EC888E042
:1065B0000E94CF0D882309F4B2CF40915A038FEF88
:1065C000840F823028F085E0433019F489E101C05E
:1065D00084E190E02091580330915903281739073E
:1065E00050F48DEF91E00E947A1864E08EE690E01E
:1065F0000E94791994CF411109C0609136015091E0
:106600003501651718F085E092E0EDCF281B390BB6
:10661000309359032093580341110FC00E94630A1D
:106620008FE991E00E947A1824E040E456E063E0AC
:106630008CE494E00E94E21872CF413041F48091E2
:1066400025018F5F809325018AE092E0EBCF4230F5
:1066500041F480915B038F5F80935B0381E192E063
:10666000E1CF809135018E5F809335010E94630AEE
:1066700088E192E0D7CF863009F0C9C080E80E9457
:10668000CF0D811105C080E20E94CF0D882379F0E3
:1066900080915E0390E0029663E070E00E944137D3
:1066A00080935E0362E08CEB92E00E94791980E1B6
:1066B0000E94CF0D811105C080E40E94CF0D882378
:1066C00079F080915E0390E0019663E070E00E94B3
:1066D000413780935E0362E08CEB92E00E9479196F
:1066E00088E00E94CF0D8823B1F10E94911820917B
:1066F0005C0330915D032817390708F46DC0281B2F
:10670000390B30935D0320935C03809126018F5FEA
:106710008093260180915E03811163C080912501E1
:106720008F5F809325018AE092E00E947A1825E02D
:1067300042E756E064E08CE494E00E94E2180E9494
:10674000911820915C0330915D032817390708F4F4
:106750005AC010925E030E94C61E0E949F2300E052
:106760002CE248E66CE070E08CE090E00E940C12B5
:1067700001E02CE248E66CE070E08CE090E00E94E2
:106780002E1281E0809327018093280183E290E01C
:106790009093630380936203EFE0F0E0F093610372
:1067A000E09360038EED93E10E94C811C0915E03F7
:1067B0002C2F40E067ED73E18CE10E94F8122C2F42
:1067C00041E060ED73E186E20E94F8122C2F42E076
:1067D0006AEC73E180E3E8CE10925D0310925C03F3
:1067E00094CF813041F480915B038F5F80935B0392
:1067F00081E192E09ACF809135018E5F80933501DF
:1068000088E192E092CF83E080936C03A4CF88E08C
:106810000E94CF0D882329F010925F0382E08093BD
:106820006C0384E00E94CF0D882319F081E08093EF
:106830006C03409168035091690360916A03709101
:106840006B038091640390916503A0916603B091FE
:10685000670384179507A607B70760F4409364039E
:1068600050936503609366037093670380E190E043
:106870000E9471340E94BA0D81E0809328012AE0C1
:1068800030E0309363032093620386E190E09093BD
:1068900061038093600381EF93E10E94C811E6E1F8
:1068A000F0E0F0936303E09362032CE230E0309376
:1068B00061032093600384EE93E1C8C981FDB6CCE7
:1068C00060E0C0E0B7CCF999FECF92BD81BDF89AE7
:1068D000992780B50895A6E1B0E044E050E00C941B
:1068E0008D340396272F0E949C340E949B34252FC1
:1068F0000E949C34242F0C949C34262FF999FECFAF
:106900001FBA92BD81BD20BD0FB6F894FA9AF99ACC
:106910000FBE01960895DC01CB01FC01F999FECF71
:1069200006C0F2BDE1BDF89A319600B40D92415017
:106930005040B8F70895262FF999FECF92BD81BD3A
:10694000F89A019700B4021639F01FBA20BD0FB6AD
:10695000F894FA9AF99A0FBE0895052E97FB1EF443
:1069600000940E94C43457FD07D00E94D73407FC1E
:1069700003D04EF40C94C434509540953095219535
:106980003F4F4F4F5F4F089590958095709561955B
:106990007F4F8F4F9F4F08950E94F934A59F900D10
:1069A000B49F900DA49F800D911D11240895A1E224
:1069B0001A2EAA1BBB1BFD010DC0AA1FBB1FEE1F79
:1069C000FF1FA217B307E407F50720F0A21BB30BC4
:1069D000E40BF50B661F771F881F991F1A9469F740
:1069E00060957095809590959B01AC01BD01CF019C
:1069F0000895A29FB001B39FC001A39F700D811D98
:106A00001124911DB29F700D811D1124911D0895B7
:106A10005058BB27AA270E9420350C946A360E9442
:106A20005C3638F00E94633620F039F49F3F19F449
:106A300026F40C9459360EF4E095E7FB0C9453368B
:106A4000E92F0E947B3658F3BA1762077307840751
:106A5000950720F079F4A6F50C949D360EF4E09598
:106A60000B2EBA2FA02D0B01B90190010C01CA0108
:106A7000A0011124FF27591B99F0593F50F4503EB3
:106A800068F11A16F040A22F232F342F4427585FA5
:106A9000F3CF469537952795A795F0405395C9F7BD
:106AA0007EF41F16BA0B620B730B840BBAF0915075
:106AB000A1F0FF0FBB1F661F771F881FC2F70EC014
:106AC000BA0F621F731F841F48F4879577956795E7
:106AD000B795F7959E3F08F0B0CF9395880F08F0D3
:106AE0009927EE0F9795879508950E9489350C9404
:106AF0006A360E94633658F00E945C3640F029F4F2
:106B00005F3F29F00C94533651110C949E360C942F
:106B100059360E947B3668F39923B1F3552391F3DC
:106B2000951B550BBB27AA2762177307840738F0FC
:106B30009F5F5F4F220F331F441FAA1FA9F335D059
:106B40000E2E3AF0E0E832D091505040E695001C0D
:106B5000CAF72BD0FE2F29D0660F771F881FBB1FC7
:106B6000261737074807AB07B0E809F0BB0B802DA5
:106B7000BF01FF2793585F4F3AF09E3F510578F0D1
:106B80000C9453360C949E365F3FE4F3983ED4F356
:106B9000869577956795B795F7959F5FC9F7880FA5
:106BA000911D9695879597F90895E1E0660F771FF7
:106BB000881FBB1F621773078407BA0720F0621B88
:106BC000730B840BBA0BEE1F88F7E09508950E94B3
:106BD000833688F09F5798F0B92F9927B751B0F0B6
:106BE000E1F0660F771F881F991F1AF0BA95C9F751
:106BF00014C0B13091F00E949D36B1E008950C941C
:106C00009D36672F782F8827B85F39F0B93FCCF3CE
:106C1000869577956795B395D9F73EF490958095CD
:106C2000709561957F4F8F4F9F4F0895E89409C0ED
:106C300097FB3EF490958095709561957F4F8F4FAF
:106C40009F4F9923A9F0F92F96E9BB279395F695C5
:106C5000879577956795B795F111F8CFFAF4BB0F43
:106C600011F460FF1BC06F5F7F4F8F4F9F4F16C0A7
:106C7000882311F096E911C0772321F09EE8872F31
:106C8000762F05C0662371F096E8862F70E060E0ED
:106C90002AF09A95660F771F881FDAF7880F969566
:106CA000879597F9089597F99F6780E870E060E00D
:106CB00008959FEF80EC089500240A941616170695
:106CC00018060906089500240A94121613061406DD
:106CD00005060895092E0394000C11F4882352F040
:106CE000BB0F40F4BF2B11F460FF04C06F5F7F4FF8
:106CF0008F4F9F4F089557FD9058440F551F59F0DF
:106D00005F3F71F04795880F97FB991F61F09F3F98
:106D100079F087950895121613061406551FF2CFC1
:106D20004695F1DF08C0161617061806991FF1CF11
:106D300086957105610508940895E894BB27662738
:106D40007727CB0197F908950E94B7360C946A36DD
:106D50000E945C3638F00E94633620F0952311F0D3
:106D60000C9453360C94593611240C949E360E9480
:106D70007B3670F3959FC1F3950F50E0551F629FCE
:106D8000F001729FBB27F00DB11D639FAA27F00D84
:106D9000B11DAA1F649F6627B00DA11D661F829FAB
:106DA0002227B00DA11D621F739FB00DA11D621F90
:106DB000839FA00D611D221F749F3327A00D611DAD
:106DC000231F849F600D211D822F762F6A2F11248F
:106DD0009F5750409AF0F1F088234AF0EE0FFF1FC2
:106DE000BB1F661F771F881F91505040A9F79E3F19
:106DF000510580F00C9453360C949E365F3FE4F3BB
:106E0000983ED4F3869577956795B795F795E7956E
:106E10009F5FC1F7FE2B880F911D9695879597F977
:106E20000895DB018F939F930E94CC34BF91AF9163
:106E3000A29F800D911DA39F900DB29F900D1124D4
:106E40000895991B79E004C0991F961708F0961BC6
:106E5000881F7A95C9F780950895AA1BBB1B51E13D
:106E600007C0AA1FBB1FA617B70710F0A61BB70BBA
:106E7000881F991F5A95A9F780959095BC01CD015F
:106E8000089597FB072E16F4009407D077FD09D0DC
:106E90000E942D3707FC05D03EF4909581959F4FB9
:106EA0000895709561957F4F08950E94F934B7FF5A
:106EB0000895821B930B0895EE0FFF1F0590F49128
:086EC000E02D0994F894FFCFC6
:106EC800262052D0262052D02000000000000000CA
:106ED80000000000000000000000102DFFFF04016A
:106EE80001010403FF01010101FFFFFFFF00E100B1
:106EF80000000000000605000008008000380016A9
:106F0800000D0054002A002A0014002C001B003831
:106F1800001A0010000C00000100FFFF0001000033
:106F2800C1808100000000000000880BF30CA90B51
:106F38009E0BEF0BAD0BCB0B000000001511780D6D
:106F48008A228922424C4F434B0048495421004D24
:106F58004F4220315354002B3120434F494E0048B3
:106F680045414C00474554204B4559004C4F434B35
:106F7800454400444545500057414C4C002B434F75
:106F8800494E004556414445004D4F5254004E4F1E
:106F980020535043004E4F20454E004D4147494332
:106FA8000053574F524400535445414C0041544BF1
:106FB800004D49535321004352495421004E4F205C
:106FC800434F494E0046554C4C0041544B205550B8
:0E6FD8000044454620555000485020555000BA
:00000001FF
